:10000000CAEF24F000000000000000000000000023
:100010000000000000000000F711000000000000D8
:1000200000000000000000000000000000000000D0
:100030000000000000000000000000000000251289
:100040000000000000000000DD15000000000000BE
:1000500000000000000000000000000000000000A0
:100060000000000000000000000000000000000090
:100070000000000000000000F41500000000000077
:100080000000000000000000000000000000000070
:100090000000000000000000000000000000000060
:0C00A00000000000000000000000000054
:0C00AC00000E3D01E1BF010E006E1200CD
:0C00B800000E3D01F9BF010E006E1200A9
:0400C400F9DF12004E
:0400C800F1DF120052
:1000CC00FBDF005202E10000FBD760006FFCEAFD91
:0200DC00120010
:1000DE00F4DF005202E10000FBD760006FFCD2FD9E
:0200EE001200FE
:0800F0001AC31BF3EBDF120041
:0800F8001AC31BF3F0DF120034
:080100001AC31BF3ECDF12002F
:080108001AC31BF3DFDF120034
:10011000D250026ED29E0500FF6A0150FE6E005062
:08012000FD6E02BED28E12003A
:100128000B840BAE9FEF00F0010E036E026A016AAA
:0A013800006A0A360232FF0E1200C0
:080142000AAE029E000E12003D
:10014A000B820BAEAFEF00F003680268016800682B
:08015A000A360232FF0E12000A
:0E016200026A016A006A086A036A000E12004F
:1001700060002FFAE1FF600033FAE2FF600067FCE5
:0E018000E6FF89C200F08AC201F0C2DF120061
:10018E000B800BAED3EF00F0026A0AAEFF0E026ECA
:0C019E00016E006E0A360232FF0E1200E5
:1001AA000A6A0350D8A40A800750D8A40A820A50BF
:1001BA00D8B438EF01F0030AD8B4F1EF00F00AB06E
:1001CA00ECEF00F006AE36EF01F034EF01F002AECC
:1001DA0034EF01F036EF01F00250800B0A6E029EF6
:1001EA000650800B069E0A18D8B402EF01F00A5096
:1001FA00D8B434EF01F036EF01F00750035CD8B4FD
:10020A000CEF01F0D8A028EF01F02EEF01F0065014
:10021A00025CD8B416EF01F0D8A028EF01F02EEF57
:10022A0001F00550015CD8B420EF01F0D8A028EF06
:10023A0001F02EEF01F00450005CD8B438EF01F061
:10024A00D8B02EEF01F00A52D8B436EF01F034EFED
:10025A0001F00A52D8B434EF01F036EF01F0D88039
:0E026A001200D8901200D880D8841200120022
:100278000301186B600057FCE9FF60005BFCEAFFB4
:100288006F00B8FF17F31751000A0FE017C319F3EF
:100298006BDF0301182B18511525E96E000E162186
:0C02A800EA6E6F00B8FF17F3EED71200EB
:0E02B400550E3A01BF6FAA0EBF6FBF81120038
:1002C2000CB0A3EF01F00CA249EF02F00E6A000E8F
:1002D2000264BAEF01F0F00E0214D8A485EF01F027
:1002E200023A01380F0B02260138F00B016E00387A
:1002F2000F0B01260038F00B006E08380F0B00269A
:100302000838F00B086E0E84D89002BE9EEF01F002
:1003120008360036013602360E2A02BE9EEF01F082
:1003220008360036013602360E2A02BE9EEF01F072
:1003320008360036013602360E2A0E5003643FEFAD
:1003420002F0035E0BBC08AE44EF02F0D880800ED0
:1003520008640030000E002201220222D8A044EFDD
:1003620002F0023201320032034A49EF02F044EF56
:1003720002F001C002F000C001F008C000F0086AFB
:10038200000E0E860264F1EF01F0F00E0214D8A402
:10039200D9EF01F0023A01380F0B02260138F00BB7
:1003A200016E00380F0B01260038F00B006E0E8430
:1003B200D89002BE9EEF01F00036013602360E2AB8
:1003C20002BE9EEF01F00036013602360E2A02BE50
:1003D2009EEF01F00036013602360E2A9EEF01F042
:1003E20001C002F000C001F0006A000E0E960E88F5
:1003F20002641EEF02F0F00E0214D8A409EF02F01C
:10040200023A01380F0B02260138F00B016E0E84FE
:10041200D89002BE9EEF01F0013602360E2A02BECD
:100422009EEF01F0013602360E2A02BE9EEF01F067
:10043200013602360E2A9EEF01F001C002F0016A77
:10044200000E0E8602644EEF02F0F00E0214D8A4E3
:100452002DEF02F0023A0E84D89002BE9EEF01F018
:1004620002360E2A02BE9EEF01F002360E2A02BEAC
:100472009EEF01F002360E2A9EEF01F0010E0C6E85
:1004820052DE51EF02F0020E0C6E5ADE51EF02F014
:10049200040E0C6E59DE51EF02F0080E0C6E60DE97
:0204A200120046
:1004A400600057FCE9FF60005BFCEAFFEE500301CB
:1004B400171905E115C300F016C301F013D015C3D5
:1004C40000F016C301F0154B162B600003F0E9FF92
:1004D400600007F0EAFF6F00B8FF00F00052E0E1AF
:0604E400006A016A12002B
:1004EA000B6A0C6A0A6A086A0350D8B4FDEF02F074
:1004FA00028E9E0E035E03BE88EF02F0D8B488EF28
:10050A0002F0EDEF02F0036C080E035CD8A0BAEF1C
:10051A0002F0036E083600C008F001C000F002C005
:10052A0001F0026A080E035CD8A0BAEF02F0036E6B
:10053A00083600C008F001C000F0016A080E035C2A
:10054A00D8A0BAEF02F0036E083600C008F0006ABD
:10055A00080E035CD8A0BAEF02F0036E0836086AE8
:10056A000350D8A4D890C6EF02F00350D8B4C6EF0F
:10057A0002F0D8900232013200320832032EBEEF66
:10058A0002F00BBC08A0D7EF02F0D8A0D7EF02F018
:10059A00082AD8B4002AD8B4012AD8B4022A02BE3A
:1005AA0001EF03F00AAEFDEF02F0021E011E001E6B
:1005BA00081E082AD8B4002AD8B4012AD8B4022AB4
:1005CA00FDEF02F0026A016A006A086AFDEF02F0B2
:1005DA000B800BAE06EF03F0026A0AAE06EF03F0D9
:1005EA00026E016E006E086E0A36023206EF03F0E2
:1005FA00000E0C6A07EF03F0010E0C6EC3DD07EF65
:10060A0003F0FF0E0250036E0150026E0050016E9D
:06061A000850006E120002
:10062000086A096A000E0762036498EF03F002503B
:1006300006180A6E075003267E0ED8A026EF03F098
:10064000035ED8B09CEF03F02AEF03F0035ED8A05E
:10065000A0EF03F0028E068E02C00EF001C00BF078
:1006600000C00DF0005004026F00D0FF0CF00150EC
:1006700005026F00D0FF00F06F00CCFF08F004020D
:10068000F3500C26F4500822000E00220D500502F3
:10069000F3500C26F4500822000E002202500402EF
:1006A000F3500826F450002202500502016A000EA1
:1006B0000122F3500026F45001220D500602F3509F
:1006C0000826F4500022026A000E012202220B507A
:1006D0000602F3500026F4500122000E02220E50B2
:1006E0000602F3500126F450022202BE80EF03F00E
:1006F00008360036013602360306D8B4A0EF03F000
:1007000093EF03F0D880800E08640030000E0022C2
:1007100001220222D8A093EF03F00232013200320C
:10072000034A9CEF03F00AAE029E000EA2EF03F014
:10073000010E17DDA2EF03F0020E07DDA2EF03F0BA
:06074000040EF2DC1200C1
:10074600D29E3901E585550EE66FAA0EE66FE58362
:0207560012008F
:0E075800550E3A01BF6FAA0EBF6FBF9112007F
:1007660010C300F00032009E0032009E0032009E50
:100776000032009EB10E0024F66E650EF76E000E76
:10078600F722000EF86E000EF82209006F00D4FF63
:1007960000F0600047FCE1FF60004BFCE2FF6000F8
:1007A60003F0E6FF010E03011125E16E000E122192
:1007B600E26E0F0E1015006EB10E0024F66E650E79
:1007C600F76E000EF722000EF86E000EF8220900F2
:1007D6006F00D4FF00F0600003F0E6FF020E112563
:1007E600E16E000E1221E26E0FC300F00032009E91
:1007F6000032009E0032009E0032009EB10E0024A0
:10080600F66E650EF76E000EF722000EF86E000EFD
:10081600F82209006F00D4FF00F0600003F0E6FF45
:10082600030E1125E16E000E1221E26E0F0E0F155A
:10083600006EB10E0024F66E650EF76E000EF722FE
:10084600000EF86E000EF82209006F00D4FF00F0CB
:10085600600003F0E6FF040E1125E16E000E122182
:06086600E26EE66A1200DA
:10086C00220E0C6E086A096A0A6A0B6A0C06D8B466
:10087C001FD0D8900B320A320932083203320232BE
:10088C0001320032D8A0F2D70C06D8B409D00450EB
:10089C0008260550092206500A2207500B22EAD7D7
:1008AC00045008260550092206500A2207500B2234
:0208BC00120028
:1008BE0003010F51170802E2006A0FD31051000A0C
:1008CE00D8A4B1D0125301E040DF60D0600047FCE5
:1008DE0000FAA5D0600047FC01FAA1D0600047FCE9
:1008EE0002FA9DD0600047FC03FA99D0600047FCE5
:1008FE0004FA95D0600047FC05FA91D0600047FCE1
:10090E0006FA8DD0600047FC07FA89D0600047FCDC
:10091E0008FA85D0600047FC09FA81D0600047FCD8
:10092E000AFA7DD0600047FC0BFA79D0600047FCD4
:10093E000CFA75D0600047FC0DFA71D0600047FCD0
:10094E000EFA6DD0600047FC0FFA69D0600047FCCC
:10095E0010FA65D0600047FC11FA61D0600047FCC8
:10096E0012FA5DD0600047FC13FA59D0600047FCC4
:10097E0014FA55D0600047FC15FA51D0600047FCC0
:10098E0016FA4DD0600047FC17FA49D003010F51FB
:10099E00000A9CE00F51010A9DE00F51020A9EE0F1
:1009AE000F51030A9FE00F51040AA0E00F51050AF0
:1009BE00A1E00F51060AA2E00F51070AA3E00F5162
:1009CE00080AA4E00F51090AA5E00F510A0AA6E091
:1009DE000F510B0AA7E00F510C0AA8E00F510D0A98
:1009EE00A9E00F510E0AAAE00F510F0AABE00F510A
:1009FE00100AACE00F51110AADE00F51120AAEE031
:100A0E000F51130AAFE00F51140AB0E00F51150A3F
:100A1E00B1E00F51160AB2E00F51170AB3E003010D
:100A2E00125301E040DC03011051010AD8A452D147
:100A3E00125301E08ADEA4D060003FFCC0FA45D11B
:100A4E0060003FFCC1FA41D160003FFCC2FA3DD1CB
:100A5E0060003FFCC3FA39D160003FFCC4FA35D1C7
:100A6E0060003FFCC5FA31D160003FFCC6FA2DD1C3
:100A7E0060003FFCC7FA29D160003FFCC8FA25D1BF
:100A8E0060003FFCC9FA21D160003FFCCAFA1DD1BB
:100A9E0060003FFCCBFA19D160003FFCCCFA15D1B7
:100AAE0060003FFCCDFA11D160003FFCCEFA0DD1B3
:100ABE0060003FFCCFFA09D160003FFCD0FA05D1AF
:100ACE0060003FFCD1FA01D160003FFCD2FAFDD0AC
:100ADE0060003FFCD3FAF9D060003FFCD4FAF5D0A9
:100AEE0060003FFCD5FAF1D060003FFCD6FAEDD0A5
:100AFE0060003FFCD7FAE9D060003FFCD8FAE5D0A1
:100B0E0060003FFCD9FAE1D060003FFCDAFADDD09C
:100B1E0060003FFCDBFAD9D060003FFCDCFAD5D098
:100B2E0060003FFCDDFAD1D060003FFCDEFACDD094
:100B3E0060003FFCDFFAC9D060003FFCE0FAC5D090
:100B4E0060003FFCE1FAC1D060003FFCE2FABDD08C
:100B5E0060003FFCE3FAB9D060003FFCE4FAB5D088
:100B6E0060003FFCE5FAB1D060003FFCE6FAADD084
:100B7E0060003FFCE8FAA9D060003FFCE9FAA5D07E
:100B8E0003011151000AD8B457D71151010AD8B434
:100B9E0057D71151020AD8B457D71151030AD8B4F6
:100BAE0057D71151040AD8B457D71151050AD8B4E2
:100BBE0057D71151060AD8B457D71151070AD8B4CE
:100BCE0057D71151080AD8B457D71151090AD8B4BA
:100BDE0057D711510A0AD8B457D711510B0AD8B4A6
:100BEE0057D711510C0AD8B457D711510D0AD8B492
:100BFE0057D711510E0AD8B457D711510F0AD8B47E
:100C0E0057D71151100AD8B457D71151110AD8B469
:100C1E0057D71151120AD8B457D71151130AD8B455
:100C2E0057D71151140AD8B457D71151150AD8B441
:100C3E0057D71151160AD8B457D71151170AD8B42D
:100C4E0057D71151180AD8B457D71151190AD8B419
:100C5E0057D711511A0AD8B457D711511B0AD8B405
:100C6E0057D711511C0AD8B457D711511D0AD8B4F1
:100C7E0057D711511E0AD8B457D711511F0AD8B4DD
:100C8E0057D71151200AD8B457D71151210AD8B4C9
:100C9E0057D71151220AD8B457D71151230AD8B4B5
:100CAE0057D71151240AD8B457D71151250AD8B4A1
:100CBE0057D71151260AD8B457D71151270AD8B48D
:100CCE0057D71151280AD8B457D70301125302E04F
:100CDE005AEC01F0A8D0030110B102D0C29001D09D
:100CEE00C280F9D0030110B102D0C29201D0C282EB
:100CFE00F2D0030110B102D0C29401D0C284EBD065
:100D0E00030110B102D0C29601D0C286E4D0030115
:100D1E0010B102D0C29801D0C288DDD0030110B14B
:100D2E0002D0C29A01D0C28AD6D0030110B102D02D
:100D3E00C29C01D0C28CCFD0030110B102D0C29E92
:100D4E0001D0C28EC8D0030110B102D0C39001D021
:100D5E00C380C1D0030110B102D0C39201D0C382AF
:100D6E00BAD0030110B102D0C39401D0C384B3D062
:100D7E00030110B102D0C39601D0C386ACD00301DB
:100D8E0010B102D0C39801D0C388A5D0030110B111
:100D9E0002D0C39A01D0C38A9ED0030110B102D0F3
:100DAE00C39C01D0C38C97D0030110B102D0C39E57
:100DBE0001D0C38E90D0030110B102D0C49001D0E7
:100DCE00C48089D0030110B102D0C49201D0C48274
:100DDE0082D0030110B102D0C49401D0C4847BD060
:100DEE00030110B102D0C49601D0C48674D00301A1
:100DFE0010B102D0C49801D0C4886DD0030110B1D7
:100E0E0002D0C49A01D0C48A66D0030110B102D0B8
:100E1E00C49C01D0C48C5FD0030110B102D0C49E1B
:100E2E0001D0C48E58D003010F51000AD8B453D745
:100E3E000F51010AD8B456D70F51020AD8B459D758
:100E4E000F51030AD8B45CD70F51040AD8B45FD738
:100E5E000F51050AD8B462D70F51060AD8B465D718
:100E6E000F51070AD8B468D70F51080AD8B46BD7F8
:100E7E000F51090AD8B46ED70F510A0AD8B471D7D8
:100E8E000F510B0AD8B474D70F510C0AD8B477D7B8
:100E9E000F510D0AD8B47AD70F510E0AD8B47DD798
:100EAE000F510F0A81E00F51100A85E00F51110A00
:100EBE0089E00F51120A8DE00F51130A91E00F5184
:100ECE00140A95E00F51150A99E00F51160A9DE08C
:0C0EDE000F51170AA1E0FF0E006E120079
:0E0EEA000FC315F310C316F33CEC01F0120019
:100EF8003F013E9F0FC304F010C305F011C306F075
:100F080012C307F0000E006E000E016E700E026E26
:100F1800830E036ED5EC00F0010ED8B0000E006E03
:100F2800005248E00FC300F010C301F011C302F0F3
:100F380012C303F03F0E046E350E056E060E066EE4
:100F4800810E076E10EC03F075EC02F000C0C4F1DE
:100F580001C0C5F102C0C6F103C0C7F1C40E01014A
:100F6800BF6F010EC06F020EBF25E96E000EC021D3
:100F7800EA6E6F00A7FFE9FF6F00ABFFEAFF6F00A3
:100F8800BBFF3DFF010EBF25E96E000EC021EA6ED2
:100F98006F00A7FFE9FF6F00ABFFEAFF6F00BBFF21
:100FA8003CFF6000FFF6E9FF600003F7EAFF6F000F
:060FB800BBFF3BFF12002D
:100FBE000D0E03011A6F84EC00F00A0E03011A6F76
:060FCE0084EC00F01200AB
:100FD4000B6A0A6A096A005004026F00D0FF09F024
:100FE4006F00CCFF08F0015005026F00D0FF0BF03A
:100FF4006F00CCFF0AF000500502F3500926F450AC
:101004000A22E86A0B2201500402F3500926F45024
:101014000A22E86A0B2208C000F009C001F00AC0E5
:0810240002F00BC003F0120002
:10102C006E0094F713F36F0048FF12F3600047FC57
:10103C00E3F93F0E3901E517E585000E03010F15A5
:10104C00036E1051030B046E04C000F0016A6000C3
:10105C0003F0E1F9FF0E0F153901E06FA3EC03F07B
:10106C00E5A301D0FDD7030112BF02D0D29E01D05F
:0A107C00D28E60004FFCE5F912006F
:101086000301136B146B60003FFCE9FF600043FC37
:10109600EAFFEE521AE011C315F312C316F360000D
:1010A6003FFCE9FF600043FCEAFF6F00B8FF17F35F
:1010B60052EC02F0000E011802E1000E001805E0E5
:1010C6000F4B102B134B142BDED713C300F014C396
:0410D60001F0120013
:1010DA0060003FFCF6FF600043FCF7FF600047FC3E
:1010EA00F8FF09006F00D4FF00F0005216E060001C
:1010FA003FFCF6FF600043FCF7FF600047FCF8FF87
:10110A0009006F00D4FF1AF384EC00F0010E03010A
:0C111A000F27000E10231123DBD712005A
:10112600086A080E0C6E003408360450085ED8B003
:0E11360002D00826D89000360C2EF5D71200F5
:101144000301136B60003FFCE9FF600043FCEAFF0E
:10115400EE5219E011C315F312C316F360003FFCFD
:10116400E9FF600043FCEAFF6F00B8FF17F352EC9D
:1011740002F0000E011802E1000E001804E10F4B0A
:0C118400102B132BDFD713C300F0120058
:1011900013C300F003011307005232E060003FFC6C
:1011A000E9FF600043FCEAFFEE50000A10E0600037
:1011B0003FFCE9FF600043FCEAFF600047FCD9FF09
:1011C00060004BFCDAFFEE50DE1801E113D0600046
:1011D0003FFCE9FF600043FCEAFF600047FCD9FFE9
:1011E00060004BFCDAFFDE50EE5C006E016A000E20
:1011F000015A08D003010F4B102B114B122BC8D7EB
:06120000006A016A120001
:081206000B6A0B86FF0E1200BB
:10120E00025006180E6E086A096A0B6A03500764CC
:10121E00FAEF09F006500A6E068E028E03500B6E20
:10122E000750036E000E0B644AEF09F00B50075E79
:10123E00D8B4EBEF09F0070E0764B9EF09F0075EBB
:10124E0000C008F001C000F002C001F0026A074EB3
:10125E00EBEF09F007648EEF09F0075E00C008F0AF
:10126E0001C000F0016A074EEBEF09F007646CEF66
:10127E0009F0075E00C008F0006A074EEBEF09F0B8
:10128E00076453EF09F00AC002F005C001F004C074
:10129E0000F0086A17EF0BF0030E07645EEF09F01B
:1012AE00075E08380F0B086E074EEBEF09F0D8906B
:1012BE000832074EEBEF09F0D8900832074EEBEFED
:1012CE0009F0D8900832EBEF09F0030E07647DEFBA
:1012DE0009F0075E08380F0B086E0038F00B082671
:1012EE0000380F0B006E074EEBEF09F0D89000326E
:1012FE000832074EEBEF09F0D89000320832074E55
:10130E00EBEF09F0D89000320832EBEF09F0030E44
:10131E000764A5EF09F0075E08380F0B086E00385A
:10132E00F00B082600380F0B006E0138F00B00266C
:10133E0001380F0B016E074EEBEF09F0D89001321A
:10134E0000320832074EEBEF09F0D890013200322E
:10135E000832074EEBEF09F0D89001320032083216
:10136E00EBEF09F0030E0764D6EF09F0075E0838BD
:10137E000F0B086E0038F00B082600380F0B006EAE
:10138E000138F00B002601380F0B016E0238F00BFE
:10139E00012602380F0B026E074EEBEF09F0D890C4
:1013AE000232013200320832074EEBEF09F0D890CC
:1013BE000232013200320832074EEBEF09F0D890BC
:1013CE000232013200320832096A000E0EAEDFEF31
:1013DE000AF0081E001E011E021E082A002201220B
:1013EE000222DFEF0AF00750D8A400EF0AF017EF41
:1013FE000BF0096A02C00AF0028E068E0750035CDB
:10140E00076ED8B4D2EF0AF0070E0764A0EF0AF009
:10141E00075E0450096E0550046E0650056E066A8E
:10142E00074ED2EF0AF0070E076475EF0AF0075E5B
:10143E000450096E0550046E056A074ED2EF0AF08D
:10144E00070E076453EF0AF0075E0450096E046A34
:10145E00074ED2EF0AF0070E07643AEF0AF00AC001
:10146E0002F017EF0BF0030E076445EF0AF0075E6C
:10147E0009380F0B096E074ED2EF0AF0D8900932D9
:10148E00074ED2EF0AF0D8900932074ED2EF0AF08B
:10149E00D8900932D2EF0AF0030E076464EF0AF017
:1014AE00075E09380F0B096E0438F00B0926043855
:1014BE000F0B046E074ED2EF0AF0D89004320932A9
:1014CE00074ED2EF0AF0D89004320932074ED2EF0F
:1014DE000AF0D89004320932D2EF0AF0030E0764F4
:1014EE008CEF0AF0075E09380F0B096E0438F00B0B
:1014FE00092604380F0B046E0538F00B0426053848
:10150E000F0B056E074ED2EF0AF0D890053204325B
:10151E000932074ED2EF0AF0D89005320432093262
:10152E00074ED2EF0AF0D890053204320932D2EFCC
:10153E000AF0030E0764BDEF0AF0075E09380F0BC1
:10154E00096E0438F00B092604380F0B046E0538AB
:10155E00F00B042605380F0B056E0638F00B05262A
:10156E0006380F0B066E074ED2EF0AF0D8900632F1
:10157E00053204320932074ED2EF0AF0D890063205
:10158E00053204320932074ED2EF0AF0D8900632F5
:10159E00053204320932086A000E0EAEDFEF0AF091
:1015AE00091E041E051E061E092A042205220622F5
:1015BE00095008260450002205500122065002222E
:1015CE000EBEF6EF0AF0D8A005EF0BF00232013294
:1015DE0000320832033E05EF0BF011EF0BF0D8B0DE
:1015EE000BEF0BF0000E081E001E011E021E082A35
:1015FE000022012202220A7E0BEF0BF0010E0C6E6E
:10160E0061EC01F019EF0BF0020E0C6E61EC01F0C3
:10161E0019EF0BF0040E0C6EA5EC00F019EF0BF0A9
:06162E00000E0C6E12001C
:101634000FC302F010C303F002C000F003C001F0B6
:10164400024A032A600003F0E9FF600007F0EAFFA2
:10165400EE5201E0F1D703010F51025C006E10510C
:0E1664000358016E010E005E000E015A1200C6
:101672000C6A0E6A0250D8A452EF0BF001C002F0BD
:1016820000C001F0006A0E860250D8A452EF0BF09F
:1016920001C002F0016A0E960E880250D8B464EFBF
:1016A2000BF00E50035ED8A4D8A06AEF0BF0D890CE
:1016B20002BE70EF0BF0003601360236032E59EFF0
:1016C2000BF06AEF0BF0010E0C6EB1EC00F074EF50
:1016D2000BF0020E0C6E94EC00F074EF0BF0040EA3
:0816E2000C6EA1EC00F01200F7
:1016EA00086A096A100E0C6E01340836093604506D
:1016FA00085E0550D8A0053C095ED8B007D0045052
:10170A0008260550D8B0053C0926D890003601367F
:06171A000C2EEAD71200BC
:101720000301006B030E005D0AE200510825E16E23
:10173000000E0921E26E200EE66E002BF3D7005159
:101740000825E16E000E0921E26EE66A00070051ED
:1017500008250A6F000E09210B6F0A0E046E07C3DD
:1017600000F0E1DC08C000F0300E002660002BFC29
:10177000E1FF60002FFCE2FF600003F0E6FF0A0ECD
:10178000046E07C300F0CFDC00C007F30050000A6E
:0A17900001E102D00007DBD71200D0
:10179A0007C30FF308C310F309C311F3010E0301C2
:0817AA00126F5FEC04F0120065
:1017B20007C304F008C305F003010B510C112CE020
:1017C200010E0B5F000E0C5B04C002F005C003F0BB
:1017D200044A052A09C300F00AC301F0094B0A2B87
:1017E200600003F0E9FF600007F0EAFF60000BF021
:1017F200E1FF60000FF0E2FF6F00BBFFE6FF600059
:101802000BF0E9FF60000FF0EAFF6F00B8FF00F095
:10181200005201E101D0D0D70BC300F00CC301F09C
:10182200010E0B5F000E0C5B005001100AE060001D
:1018320013F0E1FF600017F0E2FFE66A044A052AAE
:0C184200EBD707C300F008C301F0120050
:10184E00000E0301081902E1000E071904E1D9C2C6
:10185E0007F3DAC208F30751081103E1006A016ABF
:10186E0060D060001FFCE9FF600023FCEAFF6F0000
:10187E00B8FF00F0005203E1006A016A52D007C3BC
:10188E000FF308C310F309C311F30AC312F343ECA9
:10189E0008F0075100260851012200C007F301C0CD
:1018AE0008F3600003F0E9FF600007F0EAFF6F0045
:1018BE00B8FF00F0005208E10201D96BDA6B000E9E
:1018CE00006E000E016E2DD007C30FF308C310F388
:1018DE0009C311F30AC312F32EDC000E016E075179
:1018EE0000260851012200C0D9F201C0DAF26000D0
:1018FE0003F0E9FF600007F0EAFFEE520BE0600034
:10190E0067FBE1FF60006BFBE2FFE66A0201D94B69
:10191E00DA2B03D00201D96BDA6B07C300F008C3D0
:04192E0001F01200B2
:101932005A6ABB925B6ABB945C6ABB965D6ABB984F
:02194200120091
:101944000301076B086B096B0A6B0B6B0C6B100EB6
:101954000B6F000E0C6F7F0E0F6F650E106F000E75
:10196400116F6DEC08F08C0E03010F6F640E106F95
:10197400000E116F6DEC08F0300E0101BC25006EF5
:1019840000C000F300C01AF384EC00F0DFEC07F0B1
:101994000BC30FF30CC310F300C311F316EC08F0E0
:1019A400680E0C6EE40E0D6E0D2EFED70C2EFCD7B9
:1019B40000000301076B086B800E0819006E800E8F
:1019C400005C02E1050E075DD8B09CD06A0E0F6F73
:1019D400670E106F000E116F6DEC08F0300E0301EE
:1019E40007251A6F84EC00F0B50E03010F6F670E24
:1019F400106F000E116F6DEC08F007C300F008C300
:101A040001F0003600900136003600900136200EB9
:101A14000026000E012200C00BF301C00CF300C02D
:101A24000FF301C010F3990E0301116F020E126F30
:101A3400B3EC03F0990E0F6F020E106F75EC07F004
:101A4400700E0F6F570E106F000E116F6DEC08F0D3
:101A54000301096B0A6B800E0A19006E800E005C8C
:101A640002E1040E095D36E2050E006E000E016E01
:101A740007C304F008C305F0EAEC07F0A30E002640
:101A8400010E012209510024E96E0A510120EA6E77
:101A94006F00A7FFE9FF6F00ABFFEAFF6F00B8FF1D
:101AA40000F000C000F309510B250F6F0A510C21FF
:101AB400106F00C011F316EC08F0680E0C6EE40E03
:101AC4000D6E0D2EFED70C2EFCD700000301094B22
:101AD4000A2BC1D7050E006E000E016E07C304F079
:101AE40008C305F0EAEC07F0A30E00240F6F010E03
:101AF4000120106F75EC07F0DFEC07F00301074BD2
:101B0400082B5AD7DE0E0F6F610E106F000E116F87
:101B14006DEC08F00301076B086B800E0819006E6A
:101B2400800E005C02E1050E075D30E2400E0725E1
:101B34000B6F000E08210C6F9B0E0725E96E010E3A
:101B44000821EA6E6F00A7FFE9FF6F00ABFFEAFF11
:101B5400300EEE24006E00C000F300C01AF384ECD3
:101B640000F00BC30FF30CC310F300C311F316EC16
:101B740008F0680E0C6EE40E0D6E0D2EFED70C2EC2
:101B8400FCD700000301074B082BC7D7820E0F6F49
:101B9400610E106F000E116F6DEC08F00301076BFE
:101BA400086B800E0819006E800E005C02E1050EC1
:101BB400075D30E2500E07250B6F000E08210C6FF5
:101BC400960E0725E96E010E0821EA6E6F00A7FF45
:101BD400E9FF6F00ABFFEAFF300EEE24006E00C099
:101BE40000F300C01AF384EC00F00BC30FF30CC332
:101BF40010F300C311F316EC08F0680E0C6EE40E3B
:101C04000D6E0D2EFED70C2EFCD700000301074BE2
:0A1C1400082BC7D7DFEC07F0120021
:101C1E00000E0301081902E1000E07193BE06000F7
:101C2E001FFCE9FF600023FCEAFFEE5233E009C31C
:101C3E000FF30AC310F3F7DC00C013F307C30FF35F
:101C4E0008C310F309C311F30AC312F3C8EC08F06A
:101C5E00000E011802E1000E001805E107C300F0A6
:101C6E0008C301F019D0010E03010725156F000EF0
:101C7E000821166F600027FCE9FF60002BFCEAFFCD
:101C8E006F00B8FF17F352EC02F000C007F301C06B
:0A1C9E0008F3BED7006A016A1200C5
:101CA80007C304F008C305F004C002F005C003F040
:101CB800044A052A09C300F00AC301F00301094BCD
:101CC8000A2B600003F0E9FF600007F0EAFF6000FC
:101CD8000BF0E1FF60000FF0E2FF6F00BBFFE6FFD3
:101CE80060000BF0E9FF60000FF0EAFFEE5201E040
:0C1CF800DBD707C300F008C301F01200A6
:0E1D04000201E3933901A4919491B290120070
:081D1200067E07EC09F0120047
:101D1A000201E39307C3E4F208C3E5F2CF0EB16E02
:0E1D2A002C0EB06E3901A4919481B28012008B
:101D38000301096B01015C51000A03E1BC9ABC98DC
:101D480001D0BC9A0301076B086B800E0819006E5E
:101D5800800E005C02E1030E075DD8B0A8D0FF0E2C
:101D6800C26E2AD0BA88C298150E0C6EC60E0D6EB9
:101D78000D2EFED70C2EFCD7000031D0BA8AC29A9D
:101D8800150E0C6EC60E0D6E0D2EFED70C2EFCD742
:101D9800000025D0BA8CC29C150E0C6EC60E0D6EB6
:101DA8000D2EFED70C2EFCD7000019D0BA98BA9A7F
:101DB800BA9CFF0EC26E13D0000E081902E1000E85
:101DC8000719D0E0000E081902E1010E0719D6E044
:101DD800000E081902E1020E0719DCE0E7D702013C
:101DE800E3AF5ED02A0E0C6E8D0E0D6E0D2EFED753
:101DF8000C2EFCD7000000000F0ECA14006E00C0A5
:101E080000F300C009F3020E0B6E380E0C6EAD0E17
:101E18000D6E0D2EFED70C2EFCD70B2EFAD70F0EFB
:101E2800CA14016E01C000F30150000839E2030131
:101E38000051091935E1BC88090E006E000E016ECB
:101E4800026E036E07C304F008C305F0000E08BF56
:101E5800FF0E066E076E36EC04F0350E0026620E95
:101E68000122000E022200510024F66E000E01200D
:101E7800F76E000E0220F86E6F00DBFFF6FF6F00B2
:101E8800DFFFF7FF6F00E3FFF8FF09006F00D4FFE3
:101E980084F20F0ECA14016E0150000801E2F9D74E
:101EA8000301BA98BA9ABA9C074B082B4ED712006E
:101EB80000C008F00150006E016A026A036A0B6AEA
:101EC8000C6A016A026A036A960E036E0A6A00AE19
:101ED80074EF0FF0081E001E082AD8B4002A0A8ED4
:101EE80000C001F008C000F0086A026A39EC0BF083
:021EF8001200D6
:101EFA0003010D6B0E6B07C304F008C305F009C399
:101F0A0006F00AC307F0000E006E000E016E700E96
:101F1A00026E830E036ED5EC00F0010ED8B0000EEF
:101F2A00006E005228E007C30FF308C310F309C379
:101F3A0011F30AC312F37CEC07F03F013E8F030151
:101F4A000D6B0E6B800E0E19006E800E0C19005C64
:101F5A0002E10B510D5D0CE2150E0C6EC60E0D6EF4
:101F6A000D2EFED70C2EFCD700000D4B0E2BEAD7F8
:101F7A003F013E9F19D003010D6B0E6B800E0E19A7
:101F8A00006E800E0C19005C02E10B510D5D0CE233
:101F9A00150E0C6EC60E0D6E0D2EFED70C2EFCD72E
:0A1FAA0000000D4B0E2BEAD71200C9
:101FB4000B6A0350D8B420EF10F002500A6E028E60
:101FC4008E0E035E03AE24EF10F0036C080E035C68
:101FD400D8A0FFEF0FF0036E013602C001F0026AD1
:101FE400080E035CD8A0FFEF0FF0036E0136016A00
:101FF4000350D8A4D89009EF10F00350D8B409EFD7
:1020040010F0D89002320132032E03EF10F00BBC13
:1020140001A016EF10F0D8A016EF10F0012AD8B4E2
:10202400022A02BE33EF10F00AAE39EF10F0021E9E
:10203400011E012AD8B4022A39EF10F0026A016A9B
:1020440039EF10F00B800BAE3DEF10F0026A0AAED0
:102054003DEF10F0FF0E026E016E0A3602323DEFC4
:1020640010F0010E0C6EC7EC00F03FEF10F0000E04
:102074000C6E3FEF10F0FF0E0C6E0150006E02501C
:04208400016E1200D7
:102088000450000A12E10550000A0FE10650000A48
:102098000CE10750000A09E1FF0E006EFF0E016E09
:1020A8007F0E026EFF0E036EA8D0086A096A0750F9
:1020B800D8B4EFEF10F00350D8B4F4EF10F002509A
:1020C80006180A6E028E068E0E6A02C008F001C05B
:1020D8000CF000C00DF004500D5E0550D8A0053C72
:1020E8000C5E0650D8A0063C085E086A0C6A0D6AA9
:1020F800D8A086EF10F0D8900232013200320832B0
:10210800010E0E6E0750035ED8A093EF10F07E0EFE
:102118000E240326D8B0F9EF10F099EF10F07E0ED8
:102128000E240326D8A0FEEF10F0180E0B6E0D3605
:102138000C3608360036013602360E360450005E7C
:102148000550D8A0053C015E0650D8A0063C025EAA
:1021580006340E120EA0B4EF10F00D80BFEF10F091
:10216800045000260550D8B0053C01260650D8B0CA
:10217800062802260D900B2E9BEF10F0E5EF10F0CD
:10218800D8900036013602360E360450005E0550EF
:10219800D8A0053C015E0650D8A0063C025E063475
:1021A8000E10010B0D26D8B00C2AD8B4082AD8A4D2
:1021B800E5EF10F008320C320D32032AD8B4F9EFEB
:1021C80010F00AAE089E0850026E0C50016E0D50B9
:1021D800006E01EF11F0010E03EC09F001EF11F0B0
:1021E800020EB1EC00F001EF11F0040EA5EC00F0C6
:0C21F80001EF11F0080E94EC00F0120052
:102204000B6A0A6A096A086A0E6A033408360450BB
:10221400085E0550D8A0053C095E0650D8A0063CCF
:102224000A5E0750D8A0073C0B5EE86AD8A0010EEE
:102234000E5E0336070E0C6E0334083609360A3672
:102244000B360E36045003A012D0085E0550D8A0F9
:10225400053C095E0650D8A0063C0A5E0750D8A08B
:10226400073C0B5EE86AD8A0010E0E5E11D008266A
:102274000550D8B0053C09260650D8B0063C0A26BD
:102284000750D8B0073C0B26E86AD8B0010E0E26DA
:1022940003360C2ED1D70234083609360A360B36EB
:1022A4000E36045003A012D0085E0550D8A0053C99
:1022B400095E0650D8A0063C0A5E0750D8A0073C29
:1022C4000B5EE86AD8A0010E0E5E11D008260550F8
:1022D400D8B0053C09260650D8B0063C0A2607505B
:1022E400D8B0073C0B26E86AD8B0010E0E26023699
:1022F400070E0C6E0234083609360A360B360E36D3
:10230400045002A012D0085E0550D8A0053C095E16
:102314000650D8A0063C0A5E0750D8A0073C0B5EC6
:10232400E86AD8A0010E0E5E11D008260550D8B078
:10233400053C09260650D8B0063C0A260750D8B0FA
:10234400073C0B26E86AD8B0010E0E2602360C2E86
:10235400D1D70134083609360A360B360E36045006
:1023640002A012D0085E0550D8A0053C095E0650B4
:10237400D8A0063C0A5E0750D8A0073C0B5EE86A6A
:10238400D8A0010E0E5E11D008260550D8B0053C29
:1023940009260650D8B0063C0A260750D8B0073C98
:1023A4000B26E86AD8B0010E0E260136070E0C6E15
:1023B4000134083609360A360B360E36045001A0AD
:1023C40012D0085E0550D8A0053C095E0650D8A07E
:1023D400063C0A5E0750D8A0073C0B5EE86AD8A00A
:1023E400010E0E5E11D008260550D8B0053C092612
:1023F4000650D8B0063C0A260750D8B0073C0B2636
:10240400E86AD8B0010E0E2601360C2ED1D700345E
:10241400083609360A360B360E36045001A012D09F
:10242400085E0550D8A0053C095E0650D8A0063CBD
:102434000A5E0750D8A0073C0B5EE86AD8A0010EDC
:102444000E5E11D008260550D8B0053C092606506A
:10245400D8B0063C0A260750D8B0073C0B26E86AD9
:10246400D8B0010E0E260036070E0C6E0034083666
:1024740009360A360B360E36045000A012D0085E18
:102484000550D8A0053C095E0650D8A0063C0A5E5B
:102494000750D8A0073C0B5EE86AD8A0010E0E5E78
:1024A40011D008260550D8B0053C09260650D8B0EE
:1024B400063C0A260750D8B0073C0B26E86AD8B079
:1024C400010E0E2600360C2ED1D700B00ED00450CB
:1024D40008260550D8B0053C09260650D8B0063C5D
:0C24E4000A260750D8B0073C0B26120057
:1024F0000050086E0150006E0250016E0350026ED3
:10250000036A0B6A0C6A9E0E036E0A6A020E0C6E58
:0625100061EC01F0120075
:102516006000C7FBF6FF6000CBFBF7FF6000CFFB58
:10252600F8FF09006F00D4FF00F000521FE06000C2
:10253600C7FBF6FF6000CBFBF7FF6000CFFBF8FFA1
:1025460009006F00D4FF00F06000BFFBE1FF6000F0
:10255600C3FBE2FF600003F0E6FF0201EF4BF02B46
:10256600010EF127000EF223F323D2D76000BFFB42
:0C257600E1FF6000C3FBE2FFE66A120018
:102582000201F36B050EF35D0AE2F351F125E16EF0
:10259200000EF221E26E200EE66EF32BF3D7F3511A
:1025A200F125E16E000EF221E26EE66AF307F351C5
:1025B200F125F46F000EF221F56F0A0E046E000E83
:1025C200056EEFC200F0F0C201F075EC0BF008C02E
:1025D20000F009C001F0300E00266000D3FBE1FFDD
:1025E2006000D7FBE2FF600003F0E6FF0A0E046E14
:1025F200000E056EEFC200F0F0C201F075EC0BF0B8
:1026020000C0EFF201C0F0F2000E011802E1000E6C
:0C261200001801E102D0F307CAD7120043
:10261E0001015A6B3A6A010E5B6FDFEC07F0A10EF7
:10262E0003010F6F610E106F000E116F6DEC08F04D
:10263E00B80E03010F6F630E106F000E116F6DEC6D
:10264E0008F01E0E0301076F000E086F8DEC0EF0E2
:10265E000201E39F3901A19191819CEC0EF00201E0
:10266E00E3BF03D0E3B301D0F8D7E3A308D082ECE5
:10267E000EF0090E01016F6F010E3A6E2FD002019E
:10268E00E3AF2CD0010E01015A6FBC880201E39F0B
:10269E00000E0301076F000E086F160E096F890EEC
:1026AE000A6FF40E0B6F010E0C6F20DCBC9801014B
:1026BE005C51000A03E1BC8ABC8801D0BC8A000EC2
:1026CE000301076F000E086F480E096F880E0A6F20
:1026DE00F40E0B6F010E0C6F09DCBC9A84C200F075
:0226EE001200D8
:0C26F0006F00A0F701F001C000F0120024
:1026FC000201EF6BF06BD10E03010F6F010E106F27
:10270C0075EC07F0DFEC07F0020E0301076F020E09
:10271C00086F3D0E096F000E0A6F0FEC0EF000C033
:10272C00CEF101C0CFF1000E026E0150025C02E14D
:10273C0000500008D8B094D1D10E0301076F010EE0
:10274C00086F410E096F000E0A6F0FEC0EF000C0FF
:10275C00CEF101C0CFF1000E026E0150025C02E11D
:10276C0000500008D8B0D7D0CEC107F3CFC108F3C2
:10277C00360E0301096F000E0A6F27EC0CF000C037
:10278C00CEF101C0CFF1990E0301076F020E086F55
:10279C0000C009F301C00AF354EC0EF0990E0F6F50
:1027AC00020E106F75EC07F0DFEC07F0000E010164
:1027BC00CF1902E1000ECE19D8B4ADD0300E020103
:1027CC00EF2503011A6F84EC00F0200E03011A6F41
:1027DC0084EC00F00301076B086B380E096F000ED8
:1027EC000A6F27EC0CF000C0CEF101C0CFF1990EAE
:1027FC000301076F020E086F00C009F301C00AF352
:10280C0054EC0EF0990E0F6F020E106F75EC07F072
:10281C00DFEC07F038D0050E006E000E016EEFC233
:10282C0004F0F0C205F0EAEC07F0A30E002403015B
:10283C00076F010E0120086F990E096F020E0A6FC7
:10284C00040E0B6F000E0C6FD9EC0BF060D05FD048
:10285C00060E0201EF5D006E000EF059016E9B0E2C
:10286C000024E16E010E0120E26E300E995D006EC7
:10287C006F0087FFE1FF6F008BFFE2FF600003F04A
:10288C00E6FF45D044D00201000EF01902E1000E23
:10289C00EF19C1E0000EF01902E1010EEF19BBE0D7
:1028AC00000EF01902E1020EEF19B5E0000EF0195E
:1028BC0002E1030EEF19AFE0000EF01902E1040E75
:1028CC00EF19A9E0000EF01902E1050EEF19BFE0B7
:1028DC00000EF01902E1060EEF19BAE0000EF01925
:1028EC0002E1070EEF19B4E0000EF01902E1080E38
:1028FC00EF19AEE0000EF01902E1090EEF19A8E095
:10290C00000EF01902E10A0EEF19A2E0BBD702018A
:10291C00EF4BF02B4BD7CF0E03010F6F630E106FE5
:10292C00000E116F6DEC08F00201EF6BF06B800E76
:10293C00F019006E800E005C02E1050EEF5D24E2E2
:10294C00300EEF2503011A6F84EC00F0200E03010A
:10295C001A6F84EC00F0050E006E000E016EEFC2D3
:10296C0004F0F0C205F0EAEC07F0A30E002403011A
:10297C000F6F010E0120106F75EC07F0DFEC07F004
:10298C000201EF4BF02BD3D70A0E03010F6F630E2E
:10299C00106F000E116F6DEC08F0060E0201EF6F58
:1029AC00000EF06F800EF019006E800E005C02E1DC
:1029BC000B0EEF5D32E2EFC207F3990E0301086FC5
:1029CC00020E096F90EC0BF0990E0F6F020E106F48
:1029DC0075EC07F0200E1A6F84EC00F0060E020165
:1029EC00EF5D006E000EF059016E9B0E0024E96E37
:1029FC00010E0120EA6E6F00A7FFE9FF6F00ABFF2D
:102A0C00EAFF300EEE2403011A6F84EC00F0DFECC9
:102A1C0007F00201EF4BF02BC5D7010E0101966FA9
:102A2C00010E976F010E986F010E996F010E9A6F40
:102A3C00BC6B99EC0CF003010F6B106B630E116FF8
:102A4C0016EC08F0010E3A6E010E01016D6F010ECD
:102A5C006E6F6F6BBC94A2EC0CF00101CE6BCF6B64
:102A6C00D10E0301076F010E086F5E0E096F010E88
:102A7C000A6F0FEC0EF000C0CEF101C0CFF1000ECA
:102A8C00026E0150025C02E10050000806E2BB82BB
:102A9C00010E5A6E0101CE6BCF6BD10E0301076F85
:102AAC00010E086F630E096F010E0A6F0FEC0EF02A
:102ABC0000C0CEF101C0CFF1000E026E0150025CDD
:102ACC0002E10050000805E2BB925A6A0101CE6B8C
:102ADC00CF6BD10E0301076F010E086F680E096FE3
:102AEC00010E0A6F0FEC0EF000C0CEF101C0CFF159
:102AFC00000E026E0150025C02E10050000806E27A
:102B0C00BB84010E5B6E0101CE6BCF6BD10E03014A
:102B1C00076F010E086F860E096F010E0A6F0FEC1E
:102B2C000EF000C0CEF101C0CFF1000E026E0150CC
:102B3C00025C02E10050000805E2BB945B6A0101F3
:102B4C00CE6BCF6BD10E0301076F010E086F8B0E8E
:102B5C00096F010E0A6F0FEC0EF000C0CEF101C030
:102B6C00CFF1000E026E0150025C02E10050000831
:102B7C0006E2BB86010E5C6E0101CE6BCF6BD10EF3
:102B8C000301076F010E086F900E096F010E0A6F9B
:102B9C000FEC0EF000C0CEF101C0CFF1000E026EB2
:102BAC000150025C02E10050000805E2BB965C6A31
:102BBC000101CE6BCF6BD10E0301076F010E086FB5
:102BCC00700E096F010E0A6F0FEC0EF000C0CEF103
:102BDC0001C0CFF1000E026E0150025C02E1005008
:102BEC00000806E2BB88010E5D6E0101CE6BCF6B57
:102BFC00D10E0301076F010E086F750E096F010EE0
:102C0C000A6F0FEC0EF000C0CEF101C0CFF1000E38
:102C1C00026E0150025C02E10050000805E2BB9814
:102C2C005D6A0101CE6BCF6BD10E0301076F010EF4
:102C3C00086F7A0E096F010E0A6F0FEC0EF000C0D0
:102C4C00CEF101C0CFF1000E026E0150025C02E128
:102C5C00005000080EE2780E03010F6F640E106F27
:102C6C00000E116F6DEC08F0010E01015D6FCE6B63
:102C7C00CF6BD10E0301076F010E086F300E096F79
:102C8C00010E0A6F0FEC0EF000C0CEF101C0CFF1B7
:102C9C00000E026E0150025C02E10050000817E2C7
:102CAC00C50E03010F6F660E106F000E116F6DECE9
:102CBC0008F0090E0B6E1E0E0C6EE40E0D6E0D2E32
:102CCC00FED70C2EFCD70B2EFAD70000FF00D10E2E
:102CDC000301076F010E086F380E096F010E0A6FA2
:102CEC000FEC0EF000C0CEF101C0CFF1000E026E61
:102CFC000150025C02E10050000831E2400E030179
:102D0C000F6F010E106F75EC07F0070E0101CE2549
:102D1C00E96E000ECF21EA6E6F00A7FFE9FF6F008E
:102D2C00ABFFEAFF6F00B8FF29F2300E0201295DFC
:102D3C0013E3350E295D10E2070E0101CE25E96E75
:102D4C00000ECF21EA6E6F00A7FFE9FF6F00ABFF0B
:102D5C00EAFF300EEE5CBC6F0101CE6BCF6B120044
:102D6C0002012E6B2F6B000E2F5D02E14F0E2E5DBC
:102D7C0018E2D10E2E25E16E010E2F21E26E6F00AE
:102D8C0087FFE1FF6F008BFFE2FFE66A010E2E2545
:102D9C00006E000E2F21016E00C02EF201C02FF22A
:102DAC00E2D70101D16B02012E6B2F6B0101CC6BB1
:102DBC00CD6BCE6BCF6BD06B3D01F289F96BFA6B9F
:102DCC000101CA6BCB6B3B6A3C6A390193871200D9
:102DDC006E0094F705F03F0E3901E517000E020165
:102DEC00EF15036EF051030B046E04C000F0016A82
:102DFC00600003F0E1F9FF0EEF153901E06FE5819A
:0E2E0C00600017F0E5F96E008CF700F0120080
:102E1A00160E0301076F086B130E096FCDEC0BF04A
:102E2A00170E0301076F010E086F250E096FCDEC0F
:042E3A000BF0120087
:102E3E00EFC295F2F0C296F2F1C297F2F2C298F298
:102E4E00F3C289F2F4C28AF2F5C28BF2F6C28CF2A8
:102E5E00F7C291F2F8C292F2F9C293F2FAC294F268
:102E6E00FBC28DF2FCC28EF2FDC28FF2FEC290F258
:022E7E00120040
:102E80000201F56BF66B000EF65D02E10A0EF55DD0
:102E90000BE2F551F325E16EF651F421E26E200EBE
:102EA000E66EF54BF62BEFD7F551F325E16EF651B3
:102EB000F421E26EE66A010EF55F000EF65BF55155
:102EC000F325F76FF651F421F86F0A0E046E000E29
:102ED000056E066E076EEFC200F0F0C201F0F1C29F
:102EE00002F0F2C203F002EC11F008C000F009C0D9
:102EF00001F00AC002F00BC003F0300E00266000A3
:102F0000DFFBE1FF6000E3FBE2FF600003F0E6FFB0
:102F10000A0E046E000E056E066E076EEFC200F01C
:102F2000F0C201F0F1C202F0F2C203F002EC11F0C3
:102F300000C0EFF201C0F0F202C0F1F203C0F2F201
:102F4000000E046E031808E10450021805E1045055
:102F5000011802E10050000A01E105D0010EF55F01
:082F6000000EF65BACD7120075
:102F68000201EF51390806E3300EEF5D03E3010E6D
:082F7800006E01D0006A120096
:102F80000201F551000805E3070EF66F000EF76F1A
:102F900012D0F551160805E2170EF86F000EF96F02
:102FA00006D0F551010FF86FF96B000EF923F8C246
:102FB000F6F2F9C2F7F2F6C201F3F7C202F3FA6BC6
:102FC000FB6B046A056A066A076AEFC200F0F0C28A
:102FD00001F0F1C202F0F2C203F0D5EC00F0010EF4
:102FE000D8B0000E006E00520BE06000CFFBE1FF96
:102FF0006000D3FBE2FF2D0EE66EF34BF42BF17F66
:10300000EFC204F0F0C205F0F1C206F0F2C207F020
:10301000006A016A026A036AD5EC00F0010ED8B0BA
:10302000000E006E005237E0000E046E000E056EBA
:10303000000E066E7F0E076EEFC200F0F0C201F0C8
:10304000F1C202F0F2C203F0D5EC00F0010ED8B0EC
:10305000000E006E00521FE0EFC200F0F0C201F05F
:10306000F1C202F0F2C203F0000E046E000E056E13
:10307000200E066E820E076E10EC03F000C0EFF219
:1030800001C0F0F202C0F1F203C0F2F2010EFA5FE9
:10309000000EFB5BC9D7000E046E000E056E200EFD
:1030A000066E820E076EEFC200F0F0C201F0F1C2B0
:1030B00002F0F2C203F0D5EC00F0000ED8B0010E21
:1030C000006E00521EE0000E046E000E056E200E13
:1030D000066E820E076EEFC200F0F0C201F0F1C280
:1030E00002F0F2C203F044EC10F000C0EFF201C0B5
:1030F000F0F202C0F1F203C0F2F20201FA4BFB2B34
:10310000CAD7FA51030101270201FB51030102232F
:10311000010E0201FC6F000EFD6F000E0301036F34
:10312000000E046F000E056F7F0E066F800E020109
:10313000FD19006E800E03010219005C03E10151CC
:103140000201FC5D1EE2000E046E000E056E200EF4
:10315000066E820E076E03C300F004C301F005C3C0
:1031600002F006C303F044EC10F000C003F301C00A
:1031700004F302C005F303C006F30201FC4BFD2B70
:10318000D5D7000E046E000E056E000E066E800E82
:10319000076E03C300F004C301F005C302F006C3C9
:1031A00003F044EC10F0EFC204F0F0C205F0F1C2FD
:1031B00006F0F2C207F007EC09F000C0EFF201C020
:1031C000F0F202C0F1F203C0F2F2000E046E000E43
:1031D000056E200E066E820E076ED5EC00F0000E16
:1031E000D8B0010E006E00520BE0000E0201EF6F2E
:1031F000000EF06F000EF16F7F0EF26FFA4BFB2B9B
:103200000201800EFB19006E800E005C02E1000ED0
:10321000FA5D43E26000CFFBE1FF6000D3FBE2FF19
:10322000300EE66EF34BF42B6000CFFBE1FF600045
:10323000D3FBE2FF2E0EE66EF34BF42B800E030160
:103240000219006E800E005C02E1000E015D07E2D3
:1032500001510201FA5F030102510201FB5B02010D
:10326000FF0EFC6FFF0EFD6F800EFB19006E800ECF
:10327000FD19005C02E1FC51FA5D0FE26000CFFB3A
:10328000E1FF6000D3FBE2FF300EE66EF34BF42B60
:10329000010EFC5F000EFD5BE7D7FC6BFD6B800E43
:1032A000FD19006E800E03010219005C03E101515B
:1032B0000201FC5D69E20201EFC200F0F0C201F020
:1032C000F1C202F0F2C203F0DAEC0FF000C0FEF23D
:1032D00001C0FFF2300E00266000CFFBE1FF60006E
:1032E000D3FBE2FF600003F0E6FFF34BF42BFD514C
:1032F000FB1902E1FA51FC190AE16000CFFBE1FF82
:103300006000D3FBE2FF2E0EE66EF34BF42BFEC201
:1033100000F0FFC201F05CEC0FF000C003F301C04D
:1033200004F302C005F303C006F300C004F001C0BB
:1033300005F002C006F003C007F0EFC200F0F0C2D3
:1033400001F0F1C202F0F2C203F089EC0EF000C00D
:10335000EFF201C0F0F202C0F1F203C0F2F2000E8F
:10336000046E000E056E200E066E820E076E10ECC7
:1033700003F000C0EFF201C0F0F202C0F1F203C0AE
:10338000F2F2FC4BFD2B8BD76000CFFBE1FF60001E
:08339000D3FBE2FFE66A120024
:103398000201EF510308D8A0EF6BF0510308D8A041
:1033A800F06BF00E3D01F2170201EF513D01F213EF
:1033B800300EF213F0C200F0003600900036009094
:1033C80000360090003600900050F413F38F12007E
:1033D8000201E96BEA6BEB6BEC6BED6BEE6BF00EDD
:1033E80003010F6F640E106F000E116F6DEC08F083
:1033F8000201EF6BF06BEEDC00C0E8F2680E0C6EB9
:10340800E40E0D6E0D2EFED70C2EFCD70000E8C280
:1034180007F3990E0301086F020E096F90EC0BF089
:10342800990E0F6F020E106F75EC07F0DFEC07F0C6
:10343800700E03010F6F630E106F000E116F6DECAD
:1034480008F0100E0201ED6F000EEE6F100EEF6F18
:10345800000EF06FBFDC00C0E8F2680E0C6EE40EE0
:103468000D6E0D2EFED70C2EFCD70000E8C21AF305
:1034780084EC00F0DFEC07F0300E0201E85D01019A
:10348800BC6F170E03010F6F600E106F000E116FE7
:103498006DEC08F00201E96BEA6B800EEA19006E28
:1034A800800E005C02E1050EE95DD8B09CD0630E89
:1034B80003010F6F670E106F000E116F6DEC08F0AF
:1034C800300E0201E92503011A6F84EC00F0BB0EEF
:1034D80003010F6F670E106F000E116F6DEC08F08F
:1034E800E9C200F0EAC201F0003600900136003669
:1034F80000900136200E0026000E012200C0EDF2D9
:1035080001C0EEF200C00FF301C010F3990E0301E1
:10351800116F020E126FB3EC03F0990E0F6F020ECB
:10352800106F75EC07F0700E0F6F570E106F000ECE
:10353800116F6DEC08F00201EB6BEC6B800EEC196F
:10354800006E800E005C02E1040EEB5D33E2EB518D
:10355800ED25EF6FEC51EE21F06F3CDC00C0E8F296
:10356800680E0C6EE40E0D6E0D2EFED70C2EFCD7D9
:103578000000050E006E000E016EE9C204F0EAC2FA
:1035880005F0EAEC07F0A30E0026010E0122020165
:10359800EB510024E16EEC510120E26E6F0087FFD1
:1035A800E1FF6F008BFFE2FF6000A3FBE6FFEB4B40
:1035B800EC2BC4D7050E006E000E016EE9C204F0B4
:1035C800EAC205F0EAEC07F0A30E002403010F6F2E
:1035D800010E0120106F75EC07F0DFEC07F0020117
:1035E800E94BEA2B5AD79B0E03010F6F5F0E106F42
:1035F800000E116F6DEC08F00201E96BEA6B800EAA
:10360800EA19006E800E005C02E1050EE95D35E204
:10361800400EE925006E000EEA21016E00C0EDF2B1
:1036280001C0EEF200C0EFF201C0F0F2EEEC16F0CD
:1036380000C0E8F2680E0C6EE40E0D6E0D2EFED77B
:103648000C2EFCD70000E8C21AF384EC00F09B0EA5
:103658000201E925E16E010EEA21E26E300EE85D15
:10366800006E6F0087FFE1FF6F008BFFE2FF6000D5
:1036780003F0E6FFE94BEA2BC2D7C30E03010F6F35
:103688005E0E106F000E116F6DEC08F00201E96B11
:10369800EA6B800EEA19006E800E005C02E1050EEE
:1036A800E95D35E2500EE925006E000EEA21016E53
:1036B80000C0EDF201C0EEF200C0EFF201C0F0F27E
:1036C800EEEC16F000C0E8F2680E0C6EE40E0D6E1B
:1036D8000D2EFED70C2EFCD70000E8C21AF384EC9E
:1036E80000F0960E0201E925E16E010EEA21E26E74
:1036F800300EE85D006E6F0087FFE1FF6F008BFF03
:10370800E2FF600003F0E6FFE94BEA2BC2D7DFECEB
:0437180007F01200A4
:10371C000201E86BBC88000E0301076F000E086FF6
:10372C00160E096F890E0A6FF40E0B6F010E0C6FDB
:10373C007DEC0FF0BC98BC8AFB0E03010F6F600E82
:10374C00106F000E116F6DEC08F00FEC13F000C051
:10375C0029F2BC98BC8A020129512A0AD8A4E6D0C5
:10376C00010E01015C6FC50E03010F6F5F0E106F30
:10377C00000E116F6DEC08F0240E03010F6F630E39
:10378C00106F000E116F6DEC08F04A0E03010F6FF5
:10379C00010E106F75EC07F0650E0F6F600E106F59
:1037AC00000E116F6DEC08F07F0E0201826F000E9F
:1037BC00836F2A6B2B6B0101BE51010A3DE1300E68
:1037CC0002012A2503011A6F84EC00F0700E03012C
:1037DC000F6F570E106F000E116F6DEC08F0050E89
:1037EC00006E000E016E2AC204F02BC205F0EAEC4A
:1037FC0007F0A30E002403010F6F010E0120106FC0
:10380C0075EC07F0200E1A6F84EC00F0700E0301BB
:10381C000F6F570E106F000E116F6DEC08F082C217
:10382C00EFF283C2F0F2990E0201F16F020EF26F09
:10383C00C1EC12F0DFEC07F0050E006E000E016E0D
:10384C002AC204F02BC205F0EAEC07F0A30E002408
:10385C0003010F6F010E0120106F4A0E116F010E44
:10386C00126F040E136FC8EC08F0000E011802E181
:10387C00000E001804E10201826B836B09D0020177
:10388C002A4B2B2B000E2B5D02E1050E2A5D93E3D8
:10389C00000E831902E1000E821933E1C00E030100
:1038AC000F6F610E106F000E116F6DEC08F00201BE
:1038BC002A6B2B6B000E2B5D02E1050E2A5D19E2C3
:1038CC00050E006E000E016E2AC204F02BC205F02C
:1038DC00EAEC07F0A30E002403010F6F010E012088
:1038EC00106F75EC07F0DFEC07F002012A4B2B2B65
:1038FC00E1D7DFEC07F001015C6B090E0201E86F08
:10390C0015D0BC88BC9ABC0E03010F6F620E106FF1
:10391C00000E116F6DEC08F04A0E03010F6F010ED3
:10392C00106F75EC07F0070E0201E86FE8C200F0AB
:02393C00120077
:10393E00DFEC07F04A0E03010F6F010E106F75ECEE
:10394E0007F0DFEC07F00201E86B6E0E03010F6F5C
:10395E00650E106F000E116F6DEC08F0050E006E07
:10396E00000E016EE8C204F0000E056EEAEC07F0E0
:10397E00A30E002403010F6F010E0120106F75ECD2
:10398E0007F0DFEC07F0050E006E000E016EE8C2C8
:10399E0004F0000E056EEAEC07F0A30E00240301FE
:1039AE000F6F010E0120106F4A0E116F010E126F74
:1039BE00040E136FC8EC08F0000E011802E1000EA1
:1039CE00001801E105D00201E82B050EE85DBDE30C
:0639DE00E8C200F0120037
:1039E4000201EC6BED6B7F0EEA6F000EEB6F040EC1
:1039F400586E050E016E57C000F0015004E0003609
:103A04000090FF0FFBD7040E00103F013F6F3E9F55
:103A14000201EC51EA25E96EED51EB21EA6E6F00EB
:103A2400A7FFE9FF6F00ABFFEAFF6F00B8FF29F2C1
:103A34002951FF0A01E108D0EC4BED2B000EED5D9E
:103A440002E1320EEC5DE4E3EC518025E16EED51D0
:103A54008121E26E6F0087FFE1FF6F008BFFE2FFC1
:103A6400E66A80C207F381C208F3EAC209F3EBC233
:103A74000AF3ECC20BF3EDC20CF3D9EC0BF0D10E4C
:103A84000F6F660E106F000E116F6DEC08F080C2A0
:103A94000FF381C210F375EC07F00201EC4BED2B30
:103AA400EC51EA25E96EED51EB21EA6E6F00A7FFB8
:103AB400E9FF6F00ABFFEAFF6F00B8FF29F229515D
:103AC400FF0A01E178D06000A7F83DFFEC51EA2538
:103AD400016EED51EB21026E010E0124E96E000E20
:103AE4000220EA6E6F00A7FFE9FF6F00ABFFEAFF59
:103AF4006F00B8FF29F26000A7F83CFF020E012412
:103B0400E96E000E0220EA6E6F00A7FFE9FF6F0066
:103B1400ABFFEAFF6F00B8FF29F26000A7F83BFF94
:103B2400030E0124E96E000E0220EA6E6F00A7FF67
:103B3400E9FF6F00ABFFEAFF6F00B8FF29F229C26B
:103B4400E8F2000EE96FE8C2E9F2E86B040E012422
:103B5400E96E000E0220EA6E6F00A7FFE9FF6F0016
:103B6400ABFFEAFF6F00B8FF29F22951E827000EE6
:103B7400E9233F013E8F0201826B836BE951835D30
:103B840002E1E851825D0CE2150E0C6EC60E0D6E5C
:103B94000D2EFED70C2EFCD70000824B832BEED7C4
:103BA4003F013E9F050E0201EC27000EED23295133
:103BB400FF0AD8A475D7350E03010F6F670E106F77
:103BC400000E116F6DEC08F0030E586E050E016EB9
:103BD40057C000F0015004E000360090FF0FFBD7FF
:0A3BE400030E00103F013F6F1200B6
:063BEE0078EC13F0120058
:103BF4006000A3FBE9FF6000A7FBEAFFEE5215E0BB
:103C04006000A3FBE9FF6000A7FBEAFF6000ABFBD9
:103C1400D9FF6000AFFBDAFFEE50DE1806E10201C7
:103C2400E84BE92BEA4BEB2BE3D76000A3FBE9FF5E
:103C34006000A7FBEAFF6000ABFBD9FF6000AFFBAD
:103C4400DAFFDE50EE5C006E016A000E015A1200CB
:103C540039019491050EB56EB28AB298B292B294BB
:103C6400B39EB46ACF0EB16E2C0EB06E8481000E7A
:103C74000201E51902E1000EE41904E1040EE46F07
:0E3C8400000EE56FE3933901A491B290120097
:103C92000101BE51010A1BE13A0E03010F6F5E0ED4
:103CA200106F000E116F6DEC08F0630E03010F6FC1
:103CB200610E106F000E116F6DEC08F0180E03010B
:103CC2000F6F5C0E106F000E116F6DEC08F03F016C
:103CD2003E9F3E993E91D40E0101C46F090EC56FFD
:103CE200000EC66F000EC76F000E0201DF6F400E9E
:103CF200E06F1D0EE16F8A0EE26F0101BE51010AF3
:103D020041E11B0E03010F6F5F0E106F000E116F6A
:103D12006DEC08F0C4C1EFF2C5C1F0F2C6C1F1F218
:103D2200C7C1F2F2990E0201F36F020EF46F40EC7A
:103D320017F0990E03010F6F020E106F75EC07F06A
:103D4200700E0F6F570E106F000E116F6DEC08F0B2
:103D5200DFC2EFF2E0C2F0F2E1C2F1F2E2C2F2F24D
:103D6200990E0201F36F020EF46F010EF56FC0ECB3
:103D720017F0990E03010F6F020E106F75EC07F02A
:103D8200DFEC07F0C40E0101BF6F010EC06FBE5120
:103D9200010A21E11C0E03010F6F660E106F000E67
:103DA200116F6DEC08F0C4C1EFF2C5C1F0F2C6C1EB
:103DB200F1F2C7C1F2F2990E0201F36F020EF46F33
:103DC20040EC17F0990E03010F6F020E106F75ECA5
:103DD20007F0DFEC07F0020E0101BF25E96E000ECD
:103DE200C021EA6E6F00A7FFE9FF6F00ABFFEAFF99
:103DF2006F00BBFF3DFF010EBF25E96E000EC02123
:103E0200EA6E6F00A7FFE9FF6F00ABFFEAFF6F00EA
:103E1200BBFF3CFF6000FFF6E9FF600003F7EAFF2B
:103E22006F00BBFF3BFF576A030E586EBE51010A7B
:103E3200D8A492D0160E03010F6F650E106F000EFC
:103E4200116F6DEC08F0300E58240201296F29C25F
:103E52001AF384EC00F04E0E03010F6F670E106F21
:103E6200000E116F6DEC08F0030E006E000E016E75
:103E720058C004F0000E056EEAEC07F0480E00246C
:103E8200E96E000E0120EA6E6F00A7FFE9FF6F00E6
:103E9200ABFFEAFF6F00B8FF0FF36F00B8FF10F33C
:103EA2006F00B8FF11F36DEC08F058C000F0000E7F
:103EB200016E026E036E0036009001360236033642
:103EC20000360090013602360336C80E0024F66E24
:103ED200640E0120F76E000E0220F86E6F00DBFF09
:103EE200F6FF6F00DFFFF7FF6F00E3FFF8FF090047
:103EF2006F00D4FF21F209006F00D4FF22F2090003
:103F02006F00D4FF23F209006F00D4FF24F2090EE0
:103F120003011A6F84EC00F021C2EFF222C2F0F228
:103F220023C2F1F224C2F2F2990E0201F36F020EE1
:103F3200F46F010EF56FC0EC17F0990E03010F6FCD
:103F4200020E106F75EC07F0710E0F6F670E106F97
:103F5200000E116F6DEC08F0050E016E57C000F0F7
:103F6200015004E000360090FF0FFBD758500010BC
:103F72003F013F6F0101BE51010A09E1320E030107
:103F82000F6F5B0E106F000E116F6DEC08F0C4C165
:103F920000F0C5C101F0C6C102F0C7C103F078EC60
:103FA20012F058C004F0000E056E066E076E04365D
:103FB2000490053606360736043604900536063672
:103FC2000736C80E0424F66E640E0520F76E000E46
:103FD2000620F86E6F00DBFFF6FF6F00DFFFF7FFD2
:103FE2006F00E3FFF8FF09006F00D4FF04F009003F
:103FF2006F00D4FF05F009006F00D4FF06F009003E
:104002006F00D4FF07F010EC03F0000E046E000EF8
:10401200056E000E066E940E076E44EC10F000C0A2
:1040220025F201C026F202C027F203C028F20101E4
:10403200BE51010A2FE1570E03010F6F630E106F7D
:10404200000E116F6DEC08F025C2EFF226C2F0F2FD
:1040520027C2F1F228C2F2F2990E0201F36F020EA8
:10406200F46F010EF56FC0EC17F0990E03010F6F9C
:10407200020E106F75EC07F0DFEC07F0290E0B6EE5
:10408200960E0C6E7F0E0D6E0D2EFED70C2EFCD7EB
:0A4092000B2EFAD70201E38B120097
:0E409C000101966B976B986B996B9A6B1200F3
:1040AA003A01406BCA6AC280C282C284C286C2987E
:1040BA00BA98C29ABA9AC29CBA9CC28E800E416FB2
:1040CA00506BCB6AC10EC36EFF0E516F3E01BC6BC3
:1040DA00B86BC380C38AC392BB92C394BB94C39682
:1040EA00BB96C398BB983A01606BCC6A800EC46ECB
:1040FA00FF0E616FC490BC90C482C494BC94C48601
:10410A00C498C49ABC98BC9ABC9A3E01C16BC19F20
:02411A00120091
:10411C0001015A6B040E5B6F3A6A4A0E0201EF6F93
:10412C00010EF06F920EF16F670EF26F000EF36FCF
:10413C008BEC12F001014A6BBC9ABC98190E03016E
:10414C000F6F620E106F000E116F6DEC08F0020114
:10415C00854B862B990EEF6F020EF06F640EF16F8C
:10416C00640EF26F000EF36F8BEC12F085C2EFF25F
:10417C0086C2F0F2A00E0201F16F020EF26FC1ECDA
:10418C0012F02A0EA56F300E0101BC250201A96F99
:10419C00990E03010F6F020E106F75EC07F0CAAE8B
:1041AC0009D0780E0F6F660E106F000E116F6DEC4C
:1041BC0008F009D0510E03010F6F660E106F000E40
:1041CC00116F6DEC08F0CCA60AD05E0E03010F6FD8
:1041DC00660E106F000E116F6DEC08F009D0370EE3
:1041EC0003010F6F660E106F000E116F6DEC08F06F
:1041FC00CBAA0AD0440E03010F6F660E106F000E8F
:10420C00116F6DEC08F009D09F0E03010F6F660E55
:10421C00106F000E116F6DEC08F0B80E03010F6FEC
:10422C00670E106F000E116F6DEC08F0B6EC16F007
:10423C00A19191811E0E0301076F000E086F8DEC8A
:10424C000EF00201E39F9CEC0EF0000E3C1802E114
:10425C00010E3B1804E17EEC13F03B6A3C6A020150
:10426C00E3BF03D0E3B301D0EED701015A510008EC
:10427C000FE20201E3A30CD0010E3A6E010E010114
:10428C006E6FBC510308D8A06D6B090E6F6F6CD0AC
:10429C000201E3933A6AE3AF67D0BC88E39F84C220
:1042AC00EFF2B4EC17F00050000A10E14A0EEF6F79
:1042BC00010EF06F970EF16F670EF26F000EF36F39
:1042CC008BEC12F001014A6B010E3A6E01014A0EA1
:1042DC00E16E010EE26E5A51E126D8B0E22A6F006F
:1042EC0087FFE1FF6F008BFFE2FF600013FAE6FF30
:1042FC005A2BFC0E03010F6F660E106F000E116F20
:10430C006DEC08F04A0E03010F6F010E106F75EC87
:10431C0007F0000E076F000E086F160E096F880E5F
:10432C000A6FF40E0B6F010E0C6F7DEC0FF0BC9846
:10433C0001015C51000A04E0040E5A5D01E303D054
:10434C00BC8ABC8801D0BC8A000E0301076F000E2A
:10435C00086F480E096F880E0A6FF40E0B6F010E72
:10436C000C6F7DEC0FF0BC9A0101BC51030802E20A
:10437C00010E6D6F5B515A5D04E23A50000A01E187
:04438C00E6D612005F
:1043900009006F00D7FFE6FF0006FAE10106F8E129
:0243A000120009
:1043A200A10E03010F6F620E106F000E116F6DEC04
:1043B20008F0A1C107F3990E0301086F020E096FFD
:1043C20090EC0BF0990E0F6F020E106F75EC07F068
:1043D200960EE96E010EEA6E0101A151E926D8B0EE
:1043E200EA2A6F00A7FFE9FF6F00ABFFEAFFEE507A
:1043F200010AD8A444D13A0E03010F6F650E106F63
:10440200000E116F6DEC08F0DFEC07F00101A15115
:104412000008D8B033D1050EA15DD8B02FD1A1C10B
:10442200E8F2000E0201E96F1A0E03010F6F670E28
:10443200106F000E116F6DEC08F0300E0201E825CE
:1044420003011A6F84EC00F09B0E0201E825E96E6D
:10445200010EE921EA6E6F00A7FFE9FF6F00ABFFD3
:10446200EAFF6F00B8FFEAF2000EEB6F000EEB6F8F
:10447200F5D0590EE825E96E000EE921EA6E6F00CB
:10448200A7FFE9FF6F00ABFFEAFFEE50000A35E13C
:10449200770E03010F6F670E106F000E116F6DEC38
:1044A20008F03E0E0201E825F66E670EE921F76E6E
:1044B200000EF86E000EE9BFFF0EF8226F00DBFF60
:1044C200F6FF6F00DFFFF7FF6F00E3FFF8FF090061
:1044D2006F00D4FF00F00050CB10BB6E590EE825E0
:1044E200E16E000EE921E26E6F0087FFE1FF6F00CF
:1044F2008BFFE2FF010EE66E34D0550E03010F6F03
:10450200670E106F000E116F6DEC08F03E0E020187
:10451200E825F66E670EE921F76E000EF86E000EC2
:10452200E9BFFF0EF8226F00DBFFF6FF6F00DFFF2F
:10453200F7FF6F00E3FFF8FF09006F00D4FF00F000
:10454200001E0050CB14BB6E590EE825E16E000E22
:10455200E921E26E6F0087FFE1FF6F008BFFE2FF50
:10456200E66A8CD05D0E03010F6F650E106F000EB0
:10457200116F6DEC08F03E0E0201E825F66E670E33
:10458200E921F76E000EF86E000EE9BFFF0EF82269
:104592006F00DBFFF6FF6F00DFFFF7FF6F00E3FF47
:1045A200F8FF09006F00D4FF00F00050CB10BB6E83
:1045B200590EE825E16E000EE921E26E6F0087FFD9
:1045C200E1FF6F008BFFE2FF010EE66E520E0B6EF3
:1045D2002B0E0C6E000E0D6E0D2EFED70C2EFCD780
:1045E2000B2EFAD70000850E03010F6F660E106FB7
:1045F200000E116F6DEC08F03E0E0201E825F66E1A
:10460200670EE921F76E000EF86E000EE9BFFF0E8D
:10461200F8226F00DBFFF6FF6F00DFFFF7FF6F008E
:10462200E3FFF8FF09006F00D4FF00F0001E005006
:10463200CB14BB6E590EE825E16E000EE921E26E45
:104642006F0087FFE1FF6F008BFFE2FFE66A16D083
:10465200010E3A6E090E01016F6F10D0000E0201B9
:10466200EB1902E1000EEA19D8B403D7000EEB19D8
:1046720002E1010EEA19D8B475D7EAD710D0040EB8
:1046820003010F6F650E106F000E116F6DEC08F0D5
:10469200DFEC07F0010E3A6E090E01016F6F120096
:1046A20039019791050EA26EA16A9E6A770EA06EDD
:1046B200F30E9F6E0201E38939018781A791A08ED3
:0446C20097811200CA
:1046C6000DEC17F0EE0E0201EF6F3B0EF06F000ED1
:1046D600F16F000EF26F080EF36F010EF46F1A0EF3
:1046E600F56F030EF66FFF0EF76FFF0EF86F000EF5
:1046F600F96F000EFA6FC40EFB6F000EFC6F000E12
:10470600FD6F000EFE6F1FEC17F0EF6BF06BCCEC3D
:0447160019F0120084
:10471A00A30E0201EF6F010EF06F8D0EF16F670E9F
:10472A00F26F000EF36F8BEC12F0A80E0201EF6F1E
:10473A00010EF06F830EF16F670EF26F000EF36FCA
:10474A008BEC12F0AD0E0201EF6F010EF06F880EC6
:10475A00F16F670EF26F000EF36F8BEC12F0B20E70
:10476A000201EF6F010EF06FAB0EF16F670EF26F81
:10477A00000EF36F8BEC12F0B70E0201EF6F010E11
:10478A00F06FB00EF16F670EF26F000EF36F8BECE5
:04479A0012F0120007
:1047DC000CC029F00DC028F06F0084FF32F06F0080
:1047EC0088FF33F06F00A4FF30F06F00A8FF31F0AA
:1047FC006F00CCFF2EF06F00D0FF2FF06F00D4FFB6
:10480C002DF06F00E0FF2AF06F00DCFF2BF06F0043
:10481C00D8FF2CF03901A1A114D091A112D0150E02
:10482C000C6EC60E0D6E0D2EFED70C2EFCD7000096
:10483C00CBA004D00201E38F01016D6B3901A19172
:10484C0091916000B7F0F5FF6000ABF0F8FF6000ED
:10485C00AFF0F7FF6000B3F0F6FF6000BBF0F3FFC2
:10486C006000BFF0F4FF29C00CF028C00DF0600010
:10487C00C3F0E9FF6000C7F0EAFF6000CBF0E1FF96
:08488C006000CFF0E2FF110013
:1048940000C027F001C026F03901A3A774D093A764
:1048A40072D0F7EC1DF000C0D0F13D01F9AB0FD090
:1048B400F99B010E0201DB25006E000EDC21016E66
:1048C40000C0DBF201C0DCF26F00A0F7D0F13D01C3
:1048D400F9A70FD0010E0201DB25006E000EDC21CA
:1048E400016E00C0DBF201C0DCF2F7EC1DF000C089
:1048F400D0F10101D0510A0A07E0CB51000802E1CE
:10490400CA514F0801E31FD0010E3B6E000E3C6EEE
:10491400D10E02012E25E16E010E2F21E26E6F00F1
:1049240087FFE1FF6F008BFFE2FFE66A390193978F
:104934002EC2CAF12FC2CBF102012E6B2F6B3901AB
:10494400A495949520D03B6A3C6AD10E02012E2591
:10495400E16E010E2F21E26E6F0087FFE1FF6F0011
:104964008BFFE2FF600043F7E6FF2EC2CAF12FC2BD
:10497400CBF1010E2E25006E000E2F21016E00C01A
:104984002EF201C02FF227C000F026C001F0110062
:10499400DFEC33F0600E3901D96F080EDF6F6E0063
:1049A40070F734F0000E356E55EC20F03B6A3C6A2B
:1049B4000201E393E3950101C86BC96B02012C6BFF
:1049C4002D6BE46BE56B0101BE6B0201E39B0101FE
:1049D400C46BC56BC66BC76BC40EBF6F010EC06FD3
:1049E400ACEC03F0170EE56F150EE66F260E106F94
:1049F4005AEC01F08A0E3D01F56F000EF66FF28F4E
:104A040060DEEE0E0201EF6F3B0EF06F000EF16FF1
:104A1400000EF26F080EF36F010EF46F1A0EF56FAD
:104A2400030EF66FFF0EF76FFF0EF86F000EF96FAF
:104A3400000EFA6FC40EFB6F000EFC6F000EFD6FCC
:104A4400000EFE6F1FEC17F0090E0B6E1E0E0C6E9F
:104A5400E40E0D6E0D2EFED70C2EFCD70B2EFAD7BE
:104A640000002A6B2B6B000E2B5D02E10F0E2A5DFA
:104A740010E24A0E2A25E16E010E2B21E26E6F0030
:104A840087FFE1FF6F008BFFE2FFE66A2A4B2B2BC7
:104A9400EAD72A6B2B6B000E2B5D02E13F0E2A5DD9
:104AA40010E2990E2A25E16E020E2B21E26E6F00B0
:104AB40087FFE1FF6F008BFFE2FFE66A2A4B2B2B97
:104AC400EAD72A6B2B6B000E2B5D02E14F0E2A5D99
:104AD40010E2300E2A25E16E020E2B21E26E6F00E9
:104AE40087FFE1FF6F008BFFE2FFE66A2A4B2B2B67
:104AF400EAD72A6B2B6B000E2B5D02E1050E2A5DB3
:104B040010E2590E2A25E16E000E2B21E26E6F0091
:104B140087FFE1FF6F008BFFE2FFE66A2A4B2B2B36
:104B2400EAD72A6B2B6B000E2B5D02E1050E2A5D82
:104B340010E2960E2A25E16E010E2B21E26E6F0023
:104B440087FFE1FF6F008BFFE2FFE66A2A4B2B2B06
:104B5400EAD799EC0CF03A0E03010F6F640E106F54
:104B6400000E116F6DEC08F002012A6B2B6B000E26
:104B74002B5D02E10B0E2A5D25E2030E006E000E92
:104B8400016E2AC204F02BC205F0EAEC07F05E0EB7
:104B94000024E96E000E0120EA6E6F00A7FFE9FF12
:104BA4006F00ABFFEAFF6F00B8FF0FF36F00B8FFB1
:104BB40010F36F00B8FF11F36DEC08F002012A4BFB
:104BC4002B2BD5D7DFEC07F0A10E03010F6F630E7B
:104BD400106F000E116F6DEC08F0000ECCB2010ED8
:104BE40003011A6F300E1A2784EC00F0DFEC07F093
:104BF400D76AD66A080ED56E3901A18B3D01F399A7
:104C0400F38FF289390183873D01F49DB6EC16F0E8
:104C14005B9187818191D2809191D28E0201EF6B59
:104C2400F06BEEEC16F000C0D0F1680E0C6EE40EE2
:104C34000D6E0D2EFED70C2EFCD700000101D051B5
:104C4400630A27E09E0E03010F6F470E106F000EDC
:104C5400116F6DEC08F003010F6B106B630E116F95
:104C640016EC08F0680E0C6EE40E0D6E0D2EFED7D9
:104C74000C2EFCD7000099EC0CF0D70E03010F6F3B
:104C8400600E106F000E116F6DEC08F0A2EC0CF0CA
:104C94000BD0890E03010F6F630E106F000E116F9E
:104CA4006DEC08F0ECEC19F0E10E03010F6F650EEA
:104CB400106F000E116F6DEC08F0990E0201EF6F8A
:104CC400020EF06F9C0EF16F670EF26F000EF36F21
:104CD4008BEC12F0990E03010F6F020E106F75EC3E
:104CE40007F0A30E0201E86F010EE96F990EEA6F57
:104CF400020EEB6FFAEC1DF000C0DDF201C0DEF233
:104D0400000E011802E1000E00180CE10101966B7F
:104D1400A10E03010F6F650E106F000E116F6DEC85
:104D240008F00CD04C0E03010F6F650E106F000ECF
:104D3400116F6DEC08F0010E0101966F300E020147
:104D4400806F020E816FDFEC07F02AEC1EF09F0EDD
:104D540003010F6F5C0E106F000E116F6DEC08F005
:104D640049EC1EF0F2EC1CF0010E01016D6F010E16
:104D74006E6FD60E03010F6F620E106F000E116F6F
:104D84006DEC08F08CDCBCC1DDF2000E0201DE6FBC
:104D94000101BC6B0201856B866B000E03010F6F72
:104DA400000E106F160E116F880E126F7CEC07F058
:104DB400060E0101C16F000EC26FDFEC07F00201A5
:104DC400846B010E0101BE6FC36B3A6A6F6BBD6BDE
:104DD400A06B5A6B040E5B6F4A0E0201EF6F010E5B
:104DE400F06FA10EF16F670EF26F000EF36F8BEC94
:104DF40012F001014A6BBC9ABC988DEF2BF00101B3
:104E04005C6BA06B6D6B3A6A5A6B040E5B6F000EA1
:104E140003010F6F000E106F160E116F880E126FC4
:104E24007CEC07F0480E03010F6F5D0E106F000E4F
:104E3400116F6DEC08F08EEC20F03A50000A03E19B
:104E4400010E6F6F13D002018451230A0CE11E0E70
:104E540003010F6F610E106F000E116F6DEC08F0FF
:104E640001016F6B03D00101090E6F6FB5EF2BF0D9
:104E7400EE0E03010F6F5F0E106F000E116F6DECDD
:104E840008F09FEC1CF000C0A1F1060E03010F6FA7
:104E9400670E106F000E116F6DEC08F0300E0101FB
:104EA400A12503011A6F84EC00F0050E0101A15D38
:104EB40024E2960EE96E010EEA6EA151E926D8B0FD
:104EC400EA2A6F00A7FFE9FF6F00ABFFEAFFEE508D
:104ED400010A0AE1F00E03010F6F650E106F000E58
:104EE400116F6DEC08F009D0D10E03010F6F650E40
:104EF400106F000E116F6DEC08F0DFEC07F0090E77
:104F040001016F6FA151000A02E1030E6F6F040EDD
:104F1400BC5D1CE2A151000819E2050EA15D16E278
:104F24009651010A13E1960EE96E010EEA6EA15143
:104F3400E926D8B0EA2A6F00A7FFE9FF6F00ABFFAC
:104F4400EAFFEE50010A02E1020E6F6FB5EF2BF09B
:104F54000B0E03010F6F5E0E106F000E116F6DECE0
:104F640008F00101A26BBC6B6E6B4A6BD1EC21F0B3
:104F7400BC88000E0301076F000E086F160E096F40
:104F8400890E0A6FE80E0B6F030E0C6F7DEC0FF0A9
:104F9400BC88BC8A0101BC6BA26B6F6BE4D3BC8878
:104FA400BC9AA06BB20E03010F6F600E106F000E5F
:104FB400116F6DEC08F07A0E03010F6F5D0E106F28
:104FC400000E116F6DEC08F00FEC13F000C029F225
:104FD40002012951300A0DE0040E0101BC5D08E212
:104FE40002012951300804E2350E295D01E201D0A5
:104FF40047D00201300E295D0101A06F230E030189
:105004000F6F670E106F000E116F6DEC08F029C260
:105014001AF384EC00F0DFEC07F0860E03010F6F47
:10502400620E106F000E116F6DEC08F00FEC13F0B0
:1050340000C029F2BC8A020129512A0A20E16B0E20
:1050440003010F6F620E106F000E116F6DEC08F00C
:1050540001015A6BBC88000E0301076F000E086F34
:10506400160E096F890E0A6FE80E0B6F030E0C6F94
:105074007DEC0FF0BC98BC8A040E01016F6F13D055
:1050840002012951230A0CE1FC0E03010F6F610E8A
:10509400106F000E116F6DEC08F001016F6B03D0FF
:1050A4000101090E6F6F5FD3AB0E03010F6F5D0E2D
:1050B400106F000E116F6DEC08F03BD0E50E03018C
:1050C4000F6F630E106F000E116F6DEC08F0DFECC4
:1050D40007F0060E01016F6F3DD0F20E03010F6F52
:1050E400660E106F000E116F6DEC08F0300E0101AA
:1050F400A02503011A6F84EC00F0DFEC07F0050E25
:1051040001016F6F27D0920E03010F6F660E106FAF
:10511400000E116F6DEC08F0300E0101A0250301A3
:105124001A6F84EC00F0DFEC07F0090E01016F6FD9
:1051340011D00101A051000AC1E0A051010ACDE043
:10514400A051020ACAE0A051030AC7E0A051040A10
:10515400C4E0D9D708D3140E03010F6F5D0E106F8E
:10516400000E116F6DEC08F0300E0101A025030153
:105174001A6F84EC00F0DFEC07F0DF0E03010F6F11
:105184005C0E106F000E116F6DEC08F00FEC13F055
:1051940000C029F2300E0201295D016E01C0BDF18B
:1051A4000150000A05E00101BD51010A01E053D09C
:1051B4008C0E03010F6F600E106F000E116F6DECFB
:1051C40008F00FEC13F000C029F2020129512A0A59
:1051D40041E1DC0E03010F6F640E106F000E116FBE
:1051E4006DEC08F0300E0101A02503011A6F84EC68
:1051F40000F0200E03011A6F84EC00F00101BD5190
:10520400000A0AE1AC0E03010F6F660E106F000E68
:10521400116F6DEC08F009D0900E03010F6F650E4D
:10522400106F000E116F6DEC08F0DFEC07F0BC8816
:10523400BC9A520E0B6E2B0E0C6E000E0D6E0D2EC4
:10524400FED70C2EFCD70B2EFAD70000BC8A060E14
:1052540001016F6F03D00101090E6F6F84D2710ECB
:1052640003010F6F5F0E106F000E116F6DEC08F0ED
:105274008EEC20F0DFEC07F08EEC1BF000C06FF139
:105284000101A051000A55E1410E03010F6F610EA7
:10529400106F000E116F6DEC08F0050E006E000E1D
:1052A400016EA0C104F0000E056EEAEC07F0A30E37
:1052B40000240301076F010E0120086F4A0E096FD5
:1052C400010E0A6F040E0B6F000E0C6FD9EC0BF07D
:1052D400010E01015C6F3A6A010E0201876F000E34
:1052E400886F01016D6B6E6BBC94BC6B960EE16EA6
:1052F400010EE26EA051E126D8B0E22A6F0087FFCA
:10530400E1FF6F008BFFE2FF010EE66E500E03011A
:105314000F6F000E106F310E116F16EC08F0680E4F
:105324000C6EE40E0D6E0D2EFED70C2EFCD7000075
:1053340095D00101A0510008D8B090D0050EA05D11
:10534400D8B08CD0FF0E03010F6F650E106F000EE6
:10535400116F6DEC08F0050E006E000E016EA0C119
:1053640004F0000E056EEAEC07F0A30E002403011E
:10537400076F010E0120086F4A0E096F010E0A6FB4
:10538400040E0B6F000E0C6FD9EC0BF0100E0F6FA8
:10539400640E106F000E116F6DEC08F0300E0101F9
:1053A400BD2503011A6F84EC00F09B0EE16E010E23
:1053B400E26E0101A051E126D8B0E22A6F0087FF16
:1053C400E1FF6F008BFFE2FF6000F7F6E6FF280EB7
:1053D40003010F6F650E106F000E116F6DEC08F076
:1053E4000E0E03010F6F660E106F000E116F6DEC41
:1053F40008F0300E0101A02503011A6F84EC00F0BF
:105404002A0E03010F6F660E106F000E116F6DEC04
:1054140008F0960EE16E010EE26E0101A051E12644
:10542400D8B0E22A6F0087FFE1FF6F008BFFE2FF35
:10543400010EE66EA051500F03010F6F106B000EAA
:105444001023310E116F16EC08F0680E0C6EE40E8A
:105454000D6E0D2EFED70C2EFCD700000101A051BD
:10546400040802E2090E6F6F000E0301076F000EBD
:10547400086F160E096F890E0A6FE80E0B6F030E84
:105484000C6F7DEC0FF0BC88BC8A01015C6B6E6B09
:10549400BC6B6D6B070E6F6F66D16B0E03010F6FE4
:1054A400660E106F000E116F6DEC08F00101BE5115
:1054B400010A46E1DFEC07F0DB0E03010F6F5D0E1E
:1054C400106F000E116F6DEC08F002012A6B2B6B4C
:1054D400000E2B5D02E1050E2A5D30E2050E006E22
:1054E400000E016E2AC204F02BC205F0EAEC07F0AC
:1054F400A30E002403010F6F010E0120106F75EC41
:1055040007F02E0E1A6F84EC00F09B0E02012A2580
:10551400E96E010E2B21EA6E6F00A7FFE9FF6F0011
:10552400ABFFEAFF300EEE2403011A6F84EC00F0A7
:10553400DFEC07F002012A4B2B2BCAD7DFEC07F074
:10554400A2EC0CF0F2EC1CF001016F6B0CD1DFEC5F
:1055540007F0E70E03010F6F660E106F000E116F58
:105564006DEC08F0010E0101956F010E6E6F010ED6
:105574006D6FBC985A6B0201846B0101BD6BA06B0B
:10558400C36B4A0E0201EF6F010EF06FA60EF16FAE
:10559400670EF26F000EF36F8BEC12F001014A6B91
:1055A400040EBC5DD8A0BC2B100E03010F6F000EBF
:1055B400106F300E0101BC250301116F16EC08F0C9
:1055C400680E0C6EE40E0D6E0D2EFED70C2EFCD75D
:1055D40000000101BE51010A1AE1BCC107F3990E92
:1055E4000301086F020E096F90EC0BF0B90E0F6FF8
:1055F400660E106F000E116F6DEC08F0990E03012A
:105604000F6F020E106F75EC07F0DFEC07F02C0E35
:1056140003010F6F670E106F000E116F6DEC08F031
:10562400040E0101BC5D1BE2000E03010F6F000EAE
:10563400106F160E116F880E126F7CEC07F0C10EFE
:1056440003010F6F650E106F000E116F6DEC08F003
:10565400060E0101C16F000EC26F6D6B3DD0000ECE
:1056640003010F6F000E106F160E116F890E126F6B
:105674007CEC07F0B40E03010F6F640E106F000E84
:10568400116F6DEC08F0F00E0201876F000E886F49
:1056940099EC0CF04EEC20F08DEC23F0A2EC0CF025
:1056A400BC84F00E03010F6F620E106F000E116FB9
:1056B4006DEC08F0000EBCB4010E03011A6F300E3D
:1056C4001A2784EC00F0DFEC07F0010E3A6E010EAD
:1056D40001016D6F010E6E6F6F6B45D0DFEC07F04B
:1056E400460E03010F6F670E106F000E116F6DEC05
:1056F40008F06FC107F3990E0301086F020E096FDA
:1057040090EC0BF0990E0F6F020E106F75EC07F012
:1057140001016F6B28D001016F51000AD8B401EF69
:1057240027F06F51010AD8B43AEF27F06F51020AFB
:10573400D8B40ED46F51030AD8B431D46F51040ACB
:10574400D8B4B2D46F51050AD8B405D56F51060A3E
:10575400D8B485D56F51070AD8B49FD66F51090ABA
:0C576400D8B4F5D6BBD7FFEF26F0FFD776
:1057740000C019F001C018F0390194A122D0A4A1ED
:1057840020D0800E0201E519006E800E005C02E15B
:10579400010EE45D06E2B290390194910201E383C3
:1057A4000AD0010EE45D006E000EE559016E00C0E2
:1057B400E4F201C0E5F2CF0EB16E2C0EB06E3901E9
:0C57C400A49119C000F018C001F0110001
:1057D00000C025F001C024F002C023F003C022F075
:1057E00004C021F005C020F008C01FF009C01EF061
:1057F0000AC01DF00BC01CF00CC01BF00DC01AF04D
:105800003901A7A1B3D097A1B1D0040E0101BC5DAD
:1058100028E2800E006E800EC219005C02E1C151C8
:1058200000081EE2010EC15D006E000EC259016E3D
:1058300000C0C1F101C0C2F1010EC115016EC2C1AB
:1058400002F0000E0216000E021802E1010E01180D
:1058500004E13F013E8FBC8A03D03F013E9FBC9ACA
:1058600048D0010E0201E625006E000EE721016E10
:1058700000C0E6F201C0E7F2010EE615016EE7C2D4
:1058800002F0000E0216000E021802E1010E0118CD
:1058900002E1BC8A01D0BC9A0201000E006E885160
:1058A000005C02E18751000824E2010E875D006E72
:1058B000000E8859016E00C087F201C088F2010E07
:1058C0008715016E88C202F0000E0216000E021843
:1058D00002E1010E011807E101016D51010A02E127
:1058E0003F013E8F06D001016D51010A02E13F01E7
:1058F0003E9FCCA205D001015D51010A01E032D0EA
:10590000FB0E03010F6F630E106F000E116F6DEC35
:1059100008F001015D51010A09E15C0E03010F6FFE
:10592000670E106F000E116F6DEC08F0DFEC07F0E2
:105930000101BC6B99EC0CF04EEC20F08DEC23F0E7
:10594000A2EC0CF039019791520E0B6E2B0E0C6EDF
:10595000000E0D6E0D2EFED70C2EFCD70B2EFAD797
:105960000000FF003901A791F30E9F6E25C000F0E3
:1059700024C001F023C002F022C003F021C004F0D3
:1059800020C005F01FC008F01EC009F01DC00AF0BD
:0E5990001CC00BF01BC00CF01AC00DF0110073
:1067BE0010EE34F0940E006E020E016E9E0EF66E0A
:0E67CE00590EF76E000EF86EC8EC21F01200A6
:10479E00203165726520496E6974206361722066EE
:1047AE006C61672061647265737365203078303098
:1047BE00303020454570726F6D2064696666657293
:0D47CE00656E74206465203939200D0A00E5
:0457700020202000D5
:02599E00000007
:0259A0003B00CA
:0259A2003B00C8
:0159A4000002
:0259A500000000
:0459A700456E6400E5
:0759AB00436F6461676500B2
:0F59B2007D6700DC66001067002564004F64000D
:0159C10000E5
:0159C20003E1
:0559C3000000000000DF
:1059C8005D5C00A06400695E00875B00965E00EF86
:1059D8005E00475F003E63003E6000506200D05B9F
:0159E80000BE
:1059E9004D697373696F6E20496D70FF0133B100A2
:1059F9004F0145D0004F0133B1004F0145D0004F51
:105A09000133B1004F0145D0004F0133B1004F01BF
:105A190045D0004F0133B1004F0133B1004F01456B
:105A2900D0004F01599C004F016E14004F0183A310
:105A3900004F019ADF004F019ADF009E000000012C
:105A49003C019ADF009E000000013C01E88D009EA8
:105A5900000000009E022472009E000000009E01CA
:105A69009ADF009E000000013C019ADF009E0000C1
:105A790000013C016E14009E000000009E0183A3FA
:105A8900009E000000009E019ADF009E00000001B8
:015A9900FF0D
:085A9A005265732E4D435500C7
:085AA2004D5361626F743D0079
:0A5AAA00427566666572310D0A0050
:105AB40030313233343536373839303132333400DB
:015AC40000E1
:015AC50000E0
:015AC60000DF
:015AC70000DE
:055AC80052314F4E00B9
:055ACD0052314F4600BC
:055AD20052324F4E00AE
:015AD70000CE
:015AD80000CD
:015AD90000CC
:055ADA0052344F4E00A4
:055ADF0052344F4600A7
:0C5AE4005265732E44697374616E740087
:055AF00052324F460098
:055AF50052334F4E008A
:055AFA0052334F46008D
:015AFF0000A6
:055B00000000000000A0
:055B0500000000010199
:015B0A00009A
:015B0B000099
:015B0C000098
:105B0D003030303000303030310030303032003015
:095B1D0030303300303030340028
:015B2600007E
:015B2700007D
:015B2800007C
:025B2900C401B5
:025B2B00000078
:015B2D000077
:045B2E000000000073
:105B32002043616C63756C206469726563742046EE
:105B4200303D20282028666C6F61742920496E63DD
:105B520072656D656E74202A204E434F315F436C2F
:105B62006F636B5B4E434F315F436C6F636B5F439D
:105B7200686F69785D20292F323039373135322EFE
:055B8200303B0D0A009C
:105B870020436F6E66696720626974203A2050313E
:105B9700384632374B34325F466F73635F696E74D2
:105BA70065726E655F776974685F504C4C5F363419
:105BB7004D487A5F566563746F7265645F49542E0A
:095BC7006366677363680D0A0050
:105BD000204C696173696F6E73204364657320455F
:105BE000787465726E65732076696120426C7565A4
:105BF000546F6F7468203A0D0A2044696769636FB7
:105C000064655F343030305F323031305F31303195
:085C1000312E6B776C0D0A00C8
:105C1800204E434F31206F7065726174657320693F
:105C28006E204669786564204475747920437963E9
:105C38006C65206D6F646520353025202C206469E3
:105C480076696465206279203220202850464D3DCF
:055C580030290D0A00D7
:105C5D00204469726563746F7279203A433A5C5FD0
:105C6D004D696B726F435C5F4D657350726F6A6502
:105C7D0074735F4D696B726F435C434C415649457C
:105C8D00525F31384632374B34325F323032310D5C
:025C9D000A00FB
:105C9F0020496E69742047656E657261746575720F
:105CAF00206465204672657175656E6365204E438D
:105CBF004F202C736F7274696520524330203D3E24
:105CCF002042757A7A6572207069657A6F0D0A00C5
:105CDF0020536169736972206C6520636F6465205E
:105CEF00436F6E6669672020303D3E4F4E2F4F4603
:105CFF0046206F7520313D3E4D6F6E6F737461623C
:055D0F006C650D0A00A7
:105D14000D0A20457461706520350D0A204E6F759B
:105D24007665617520636F646520646520636F6EBA
:105D340066696720706F7572206C652052656C61AE
:045D4400697320005F
:105D48000D0A20457461706520300D0A2053616981
:105D580073696520636F646520646520636F6D6D8A
:105D6800616E646520283420646967697473290D3D
:025D78000A001F
:105D7A0020417474656E7465205361697369652086
:105D8A004EB0206465204D656D6F69726520436F62
:105D9A006D6D616E6465203C3020E020343E0D0A52
:015DAA0000F8
:105DAB000D0A20457461706520340D0A2041696726
:105DBB0075696C6C616765206E6F7576656C6C656B
:105DCB0020636F6D6D616E646520706F757220005E
:105DDB00206E6F7576656C6C65206C6973746520CD
:105DEB0064652063646520736175766567617264B1
:105DFB00E96520656E20456570726F6D200D0A0098
:105E0B000D0A20457461706520320D0A20457865B6
:105E1B00637574696F6E206465206C6120436F6DD0
:0F5E2B006D616E64652052656C6169730D0A00CC
:105E3A0020496E69742064652062617365204E434F
:105E4A004F2028766F697220706167652034353477
:0F5E5A002064617461736865657429200D0A0006
:105E69002050726F6A6574203A436C617669657275
:105E79005F48545F31384632374B34325F32303203
:0D5E8900312D31302E6D637070690D0A00EF
:105E960020456570726F6D3A2020456E20466C6114
:105EA6007368204020333130203030303020E020FD
:0D5EB6003331302030334646462E0D0A00B1
:105EC3000D0A205265737469747565204574617495
:105ED300206D6F64696620636F646573203C2D2DAC
:0C5EE3002040307830303530203D200069
:105EEF0020536F75726365203A20436C6176696544
:105EFF00725F48545F31384632374B34325F32303D
:0C5F0F0032315F313031362E630D0A0054
:105F1B0020496E6372656D656E743D323531362086
:105F2B0020202D3E28666C6F61742920496E6372A8
:0C5F3B00656D656E742029203D3E20003D
:105F470020436C6176696572204D6563616E697186
:105F57007565204D617472696365203478332074E8
:0A5F67006F7563686573200D0A0072
:105F71000D0A20457461706520360D0A2053616950
:105F8100736965204E6F7576656C6C6520436F6D26
:0A5F91006D616E6465203A20200067
:105F9B000D0A20526573746974756520436F6E66C4
:105FAB006967732052656C616973203C2D2D20400D
:0A5FBB00307830303430203D2000F3
:105FC5000D0A204F4B2C205361697369652076615A
:105FD5006C6964E9652070617220546F756368654A
:095FE5002076657274650D0A0056
:105FEE000D0A2045746170652031200D0A2054651C
:105FFE0073742076616C69646974E9206465206C41
:09600E006120436465200D0A00C5
:1060170020526573746974756520436465205072F6
:106027006F67206574203420636465732052656C44
:07603700616973200D0A00EE
:10603E00204E434F206F75747075742073757220E7
:10604E00524330202D3E2042757A7A657220506977
:07605E00657A7A6F0D0A005C
:10606500206E2765737420706173207265646F6E8E
:1060750064616E74202864E96A61206166666563FF
:0760850074E929200D0A0057
:10608C00207075697320746F75636865205665722E
:10609C007465203C2A3E20706F75722076616C69A5
:0660AC006465720D0A009C
:1060B2000D0A20457461706520330D0A20456E7407
:1060C20072656520656E206D6F64652050726F6722
:0560D200722E0D0A0012
:1060D70020536175766520636F6E666967206F72FE
:1060E7006967696E616C65206465206465706172BB
:0460F700740D0A001A
:1060FB002056616C69646174696F6E2070617220E7
:10610B00546F75636865205665727465203C2A3E32
:03611B000D0A006A
:10611E000D0A20416E6E756C6174696F6E20706130
:10612E007220746F7563686520526F7567652023E2
:03613E000D0A0047
:1061410020706F7572206D6F64696620636F64657E
:106151002050726F6772616D6D6174696F6E200D91
:026161000A0032
:1061630020506F6C6172697479203D3020284E6F26
:0F6173007420696E76657274656429200D0A00C8
:106182000D0A2045746174204D6F64696620646550
:0F61920020436F6465204030783530203A20007C
:1061A10020417474656E74652031202066726170BF
:0F61B100706520636C6176696572200D0A2000AD
:1061C000204572726575722C20636F64652064656A
:0E61D0006A61206578697374616E740D0A004F
:1061DE000D0A20436F6E6669672043646520526521
:0E61EE006C616973204030783430203A200014
:1061FC000D0A20416E6E756C6174696F6E20706152
:0D620C007220746F7563686520230D0A0011
:1062190020417474656E74652034206672617070F3
:0C622900657320636C617669657220006B
:106235002E31342E372E2E2E2A2E32352E382E2E56
:0B6245002E302E33362E392E2E2E2345
:1062500020557361676520496E746572727570743C
:0B62600020566563746F72730D0A0016
:10626B00200D0A20546F756368652056657274653E
:0B627B00202A202E2E204F4B0D0A0081
:1062860020417474656E746520546F75636865206B
:0B6296005665727465202A200D0A0076
:1062A100206465636F646167652043646520656E82
:0B62B10020636F75727320203D2000F9
:1062BC00206E6F757665617520436F64616765202C
:0A62CC00616363657074E92020002F
:1062D60020496E69742054696D6572345F666F7209
:0A62E6005F416C61726D650D0A00E6
:1062F000205265706F727420416C61726D6520442C
:0A630000697374616E7465203D003E
:10630A00204E657720436F6E666967206364657304
:0A631A002052656C6169730D0A00E2
:106324002054657374207369206C65204E6F7576F4
:0A63340065617520636F6465200049
:10633E002031384632374B343220554152543120B9
:09634E003131353230300D0A0006
:1063570020526573756C7461742046726571204FA5
:0963670075747075743D2020006E
:10637000204D5361626F74616765203C2D2D202094
:096380004030783130203D20004E
:1063890020526573746974756520506172616D6519
:0863990074726167650D0A00D2
:1063A1000D0A204574617420526573657420446937
:0763B1007374616E743D007E
:1063B8002053746172742054696D656F757420334D
:0763C800207365630D0A005C
:1063CF00204E657720436F6E66696720436F646167
:0663DF006765200D0A00B5
:1063E5002041636365732050726F6772616D6D61E3
:0663F50074696F6E2E00BA
:1063FB000D0A2052455345542064697374616E74C1
:05640B0020210D0A0034
:1064100020436F6E666967204D6F64652052656C1E
:0564200061697320001A
:1064250020204D46494E544F5343202835303020C7
:056435006B487A29000C
:10643A000D0A2050726573656E746174696F6E20FF
:05644A003A200D0A00DC
:10644F00204D46494E544F53432F3420283331208B
:05645F006B487A2900E2
:10646400204964783D2A542E2E2E2E2E2A3B2A476C
:04647400302A3B008F
:106478005265736574204D43552064697374616E69
:04648800740D0A0085
:10648C00204D5361626F7461676520403078313004
:04649C00203D20007F
:1064A000204D696B726F432070726F20372E36302B
:0464B000200D0A00B1
:1064B400426C6F7175616E74652031323020736582
:0464C400630D0A005A
:1064C800002474980024749800007A8D0024749134
:0464D8000030728D91
:1064DC00204E657720436F6E6669672052656C614C
:0464EC0069732000B0
:1064F000205265616420666C6167204030783030DE
:04650000203D20001A
:10650400204E4F4E204D6F64696669E92021210DAC
:026514000A007B
:10651600204E434F31434C4B2063686F6978203DD2
:02652600200053
:1065280020616666656374E9206175737369200D7F
:026538000A0057
:10653A00204D6F64696669E965203D3E204F4B0D29
:02654A000A0045
:10654C00206D6F64696669E920202E2E4F4B0D0A71
:01655C00003E
:10655D00204F4E2070656E64616E742031730D0A8C
:01656D00002D
:10656E0020436F6D706172652061766563203A20FD
:01657E00001C
:10657F000D0A2053617576652043646573200D0AFB
:01658F00000B
:10659000206D6F6465204D6F6E6F737461626C6502
:0165A00000FA
:1065A100204E4F4E206D6F64696669E9210D0A0026
:1065B1003031323334353637383941424344454638
:1065C1006E6F6E20626C6F7175616E74650D0A007D
:1065D100204E4F4E204D6F64696669E920212100EC
:0F65E1000D0A20436F64652050726F67722000AF
:0F65F000204D6F64696669E9203D3E204F4B00E6
:0F65FF0020616666656374E9204F4B200D0A002A
:0E660E0020636F64652072656C616973200003
:0E661C0020496E6372656D656E74203D20002E
:0D662A00204D6F64696669E920210D0A00AA
:0D6637002A5252304732353542302A3B009E
:0D6644002A5052323535473042302A3B0093
:0D6651002A4C52304732353542302A3B008A
:0D665E002A5252323535473042302A3B0077
:0D666B000D0A20457461706520370D0A008E
:0D6678002A4C52323535473042302A3B0063
:0D6685002070756973204F4646200D0A00F5
:0D6692000D0A202042616420436465200051
:0D669F002A5052304732353542302A3B0038
:0D66AC00206D6F6465204F6E2F4F666600F5
:0C66B900204D5361626F746167653D0005
:0C66C5005265736574204D43550D0A00AA
:0B66D1004D656C6F646965203A200085
:0B66DC00204846494E544F5343200015
:0B66E70020457461706520390D0A0029
:0A66F2002052656C616973202300DB
:0A66FC0020436F64616765203D00D4
:0A670600202320636465203D20007D
:0A671000204C46494E544F534300FD
:09671A002052656C6169732000D6
:096723000D0A20564D656D3D0084
:09672C0020416C61726D652000D2
:09673500202E2E456E640D0A00B1
:08673E00010204081020408054
:0867460020457461706520001C
:07674E0020736F6974200045
:07675500204F46460D0A002B
:07675C0062792061697200FF
:0767630020436465202300C0
:07676A0020436465202300B9
:0667710020487A0D0A0029
:06677700204F4E0D0A0048
:06677D0020464F534300CB
:05678300303030310050
:0567880030303032004A
:05678D00303030300047
:05679200202020200082
:0567970020202020007D
:05679C00303030300038
:0567A100202020200073
:0567A60020202020006E
:0567AB00303030330026
:0567B000303030340020
:0367B50020400081
:0367B8000D0A00C7
:0367BB002040007B
:020000040030CA
:0A00000004092DA70B3F9F0F01001C
:0200000400F00A
:020000040031C9
:1000000099FFFFFFFFFFFFFFFFFFFFFFFFFFFFFF66
:1000100000FFFFFFFFFFFFFFFFFFFFFFFFFFFFFFEF
:1000200031323837313131333232323433333335A0
:1000300034343436FFFFFFFFFFFFFFFFFFFFFFFFFA
:1000400030303131FFFFFFFFFFFFFFFFFFFFFFFFFA
:100050003131313131FFFFFFFFFFFFFFFFFFFFFFB6
:10006000FFFFFFFFFFFFFFFFFFFFFFFFFFFFFFFFA0
:10007000FFFFFFFFFFFFFFFFFFFFFFFFFFFFFFFF90
:10008000FFFFFFFFFFFFFFFFFFFFFFFFFFFFFFFF80
:10009000FFFFFFFFFFFFFFFFFFFFFFFFFFFFFFFF70
:00000001FF
